:100000000C9467210C9430340C9484210C9484213A
:100010000C9484210C9482340C9484210C948421BB
:100020000C9484210C948B330C9484210C948421A3
:100030000C9484210C9484210C9441340C948421DC
:100040000C9484210C9484210C9484210C9484219C
:100050000C9484210C9484210C9484210C9484218C
:100060000C9484210C94842150474D00442E4D590A
:100070000052414400424547494E00555352007CCE
:1000800024BE248C24D9241323A524EE217E24F617
:1000900021EE215E2288228621EE21752CDC23EEC2
:1000A00021BE248C24D9241323A5242C237E245C54
:1000B00024EE215E2288223322EE21752CDC23EEF1
:1000C00021BE248C24D9241323A52446237E240274
:1000D00023EE215E2288223922EE21752CDC23EECC
:1000E00021BE248C24D9241323A5245D237E24053A
:1000F00023EE215E228822D22CEE21752CDC237D7A
:1001000024BE248C24D9241323A524EE217E240983
:1001100023EE215E228822D523EE21752CDC23EEEE
:1001200021BE248C24D9241323A52427227E241025
:1001300024EE215E2288220925EE21752CDC237B0A
:1001400024BE248C24D9241323A5242D227E2463A9
:100150002CEE215E228822F821EE21752CDC23EE84
:1001600021EE21EE21EE211323EE21CA2CEE210FE8
:1001700022EE215E22EE21EE21EE21752CEE21EE03
:1001800021BE248C24D9241323A524EE217E24927D
:1001900023EE215E2288228D23EE21752CDC23EEB6
:1001A00021BE248C24D9241323A524F4247E249D49
:1001B00023EE215E2288223F22EE21752CDC23EEE5
:1001C00021BE248C24D9241323A524E0227E24A13B
:1001D00023EE215E228822EE21EE21752CDC23EE17
:1001E00021BE248C24D9241323A52426247E2491E3
:1001F00021EE215E2288227C22EE21752CDC23EE6A
:1002000021BE248C24D9241323A524EE217E2496F8
:1002100021EE215E228822A523EE21752CDC23EE1F
:1002200021BE248C24D9241323A52495227E24FEC8
:1002300024EE215E2288222D25EE21752CDC23EE72
:1002400021BE248C24D9241323A524AC227E241B74
:1002500024EE215E2288223B24EE21752CDC23EE45
:10026000218B22BA2EAF2E1323E522BD22F422EFDA
:1002700021EE215E22EE215022EE21752CEE21206E
:100280002030202031202032202033202034202014
:1002900035202036202037202038202039202020EB
:1002A000202041202042202043202044202045209F
:1002B0002046202020202020202020202020202018
:1002C00020202020202020286929202049202020AB
:1002D00020202020202020202020313020313120DB
:1002E0003132203133203134203135203136203144
:1002F0003720313820313900207821207452744859
:100300004D74524420786C445345495347464958EC
:10031000534349454E47534C56202041202042200C
:1003200020432020442020454D41542020202020DF
:10033000202020206478794C424C48595044494D43
:1003400028692920204952455320202020202020A0
:100350002020526C49505345434C73434C50434CFE
:1003600052434C58524E2320202020202020202071
:100370005079782020202020202020204652434DF4
:10038000454D524E232020206A2C72204C520020D2
:10039000205820745020744874444720534620430A
:1003A0004620463F44454752414447445278767977
:1003B000207871204C4E4C4F47202025206B254142
:1003C0004253202020202020202020783D30202053
:1003D00020485977534E77435377544E77202070F7
:1003E00020202020202020202020202020202052DB
:1003F000544E20526E524E44434C784C5378202039
:100400002020202020202043797820202020202018
:10041000202020494E544D454D4C537820206D20CE
:10042000205320732D002020302020312020322026
:100430002033202034202035202036202037202053
:100440003820203920205C7A202020656F31306FE1
:1004500020796F312F7843485320202020202020FE
:10046000202020202A53535447544F53494E434F82
:100470005354414E45455820202020202020202044
:1004800020202D522F53475342205268786C7920F8
:100490002020454E542020202020202020202020D5
:1004A0002B204F4E20206620206753544F52434C40
:1004B000454E5420202020202E20732B0033731310
:1004C000C38382C272307010C08087C777317111C8
:1004D000C181FFC474387818C88884C5751537324F
:1004E00014341235170304050A08060BFF02090726
:1004F0000D010C00FF051A15102015051455104CA0
:10050000CC540140A02C2E400C0059260413310E6F
:10051000101333527446300A040131120C44440063
:1005200082C08CE0133130003232268C40810002D0
:100530008184023100314400014400000011D3885D
:10054000C80018480404008824C0C40484342EE27F
:10055000A2C82227C004310A301320840408304482
:10056000D0CC144D044CC8C4844442C320F0202095
:100570001004451005110F00229C0C01004C930142
:10058000C3C0091688C010123230101220444C1813
:1005900054804505985008E300850C12822404001D
:1005A0000481080D201020108844840048301186F2
:1005B000844012001133338D6080020B2911802199
:1005C0003111500404CC002413D0003333A12CA1EA
:1005D000921A0D05D040390903F284901C4D2282F5
:1005E0000DCC30D0941C068AC82C6BC3F7C01CA35A
:1005F000F079B0820010C848E88880C212108035B7
:10060000C40810115D0205A4238044804091C23BC0
:10061000E3400D02208010048E0820F33C0F1104EB
:10062000897BC35C0031001020507020E8104CA37F
:10063000024E86D6101D384C83010675CBA63C3081
:100640009EA218B0C9F318C8A030A420133138D323
:10065000915890043D8A67802003E1345D0C143486
:10066000104810B4807319D49130D31441180B1072
:10067000871C3210618C3912104C03211014241283
:10068000417DC86C18C6D7DD10121A37305E22F1D2
:100690005C08353D62563C08A248380788D825C614
:1006A00019CF15B01D152386E0862031473104D1BE
:1006B00020903F00008A0B4A50B2880150C7446224
:1006C000197210C0D8239EC4332C6D0F2A584C3C8D
:1006D000330411CB87A925A184D514303E12469846
:1006E00052837AAD1C076845A06282C03038381842
:1006F0000130070C00DC043D55320F93A104D6975E
:1007000016020EC88C8480122388B282B0AC474295
:100710000C8DC02410C633460521494812928484AA
:10072000C963904936489949236011B684C260B9BB
:1007300004650F00216433360182E1144F114098A3
:10074000B3DD4BD66A4110C33F1C845C1C43711C53
:10075000C771F12161EFA11D0F3BC0323C3F31CC8D
:10076000F21CFF073B0A9CE0107809CE3B82CE7F4B
:100770000412892028D6230D3418C34C2033033C9F
:100780004C38474C118470C70B0004111151440EB2
:10079000F0088C2050FC1189F14454344D4D2C014B
:1007A00031F4D33490D0E984818150F30F0240209A
:1007B000A3C81F42E48030F33439391981B3DC0C0B
:1007C0000183C840D3E424E132C8FC4B4C39F180AA
:1007D00001600981028A0D13010A2876F8A000FB46
:1007E000F4BF6183BF10106288E3410317AE461067
:1007F000DAF33DC7C4400400A14CCC494851C112B2
:100800000104040F218402224A481435104000E3F9
:100810000048CCA8C8E844084440A4043A20110386
:1008200012C47808442408002111000061125112FA
:10083000481810200112A445400092B24C0C100E32
:100840001081000010211011A3442160100B2A23F5
:10085000B22BA2400A502800110884028440940C54
:10086000408C00231630023112308A040E318A4443
:100870000C00A07AA30E4E1C1141844430140E5378
:10088000DD124FC411C3C44F102745C7F43C06AB5B
:1008900033314371B8C3A03A9FC16410B31BE3184E
:1008A000443162A82D974CC81148C408034062CC5B
:1008B000021D1A682023C655618B8A38CD92820C9E
:1008C000C620D4C43436B2C40535400912880A3F64
:1008D000E23BF5124C4577C794E9F60C458084A2BB
:1008E00010C85096FB202185C5EA2F1280003B706E
:1008F00074091490009582060410204400300040D2
:1009000070281403500841449841034020020C0110
:10091000B123CF49330C0311F147040D180319D249
:1009200060931803B1AA03408D070473047DE300AC
:10093000D0041110D316911431D110C300106404E7
:1009400060000CC0C0000444BE6450D086983B31A7
:100950004414330001C830018133118D99049D91F5
:10096000D38C4DE444A42C2431225111E51F0031D5
:100970000D441E533D14402160086258364414490A
:1009800013219C2C11B04C222380649F0CA1D259BE
:100990004C4CB9409574540C22183B1085DB208ACE
:1009A0000F14430418308CE84080910149018304FE
:1009B0000C1C43884C11FBA118B039099D363F72BD
:1009C00040030E31404B1253E090443E4D044140F1
:1009D000D065B218F4134352D5E38F8499DB14A683
:1009E000044C282B638C28211C1ECCC523885C7AE0
:1009F000D5A1C1CEC8013CA0000C043F3CD740406B
:100A0000C4144A00F0448004031A8AC348F101D593
:100A1000044404A2A4306B4564884411C10061C041
:100A2000E10013C11786023012274710A144CD29D7
:100A30008113A3024433340A840200012C6C50A1B8
:100A4000C7D74344C82412A082C3C5F1FC7F32FC3F
:100A5000C4E8F24444300001CC4C00109052531CC6
:100A60009D004390614CFC81311881250C84E0C4C9
:100A7000AB03315900008110440007C4344B847D1E
:100A8000158E04803411221109088210224E0013A1
:100A90000C828807190E3407583D10110B037F1084
:100AA0000B651405F30F4C4E0418420A5D0FF2AAB1
:100AB000D88B930821F5E28698C9D44074BAB274F1
:100AC000A4364D72601D19494FCFF487F04C4C4449
:100AD000401841045828180441883ADFBDBD7B1FE7
:100AE000FF3112868E0A023EC0C82155882088EA4E
:100AF0001C3B000000DC8442E8BFBF9148374A6BD2
:100B00004B7D8DAF8761917F51699947BE023EDD74
:100B100096B21346D14B58AB6E91AD6B67982C6A69
:100B2000766C0C922A725E5447099986D2B897194E
:100B300056988540C1675D570D7AA58A631A12DA07
:100B40002A0CD874DED832E7DB6CEB7E2FE6313925
:100B5000EED4101EEFED5993EB052547DBD6E45399
:100B600076D49D87EFFD49D3FB55C9FB4F19392238
:100B7000B2F4E59E073EE99CE2C49B8BC77228B4A1
:100B80000E06700EB46D112F1BE1158F2BA915F7F2
:100B90003F645012AE20682AEA98F8E672E63822DE
:100BA0001B52BEE62E8C01ECB6F4808E2E84C9401A
:100BB0001B61115FF3DE8D629D347B26164828662B
:100BC000BB36E2EF732AFAD36F2E7ACF5BC6F86694
:100BD00021F70C56578B98A2FA68044A97D16137CF
:100BE000AB4D655EDE7C007A7735BD737F3171B3C6
:100BF000C34D559F772D81639F7448462A88E2DF55
:100C00008388B0868A9864929F57CC927690228B84
:100C100093C59947970DA17F630D1D0D0694D305CC
:100C2000C614742CA2E8A87A4A74E67B777C287EE6
:100C30009AB45C7CEAC8D90996CCDC0E3E08CCCAD2
:100C400032C2C503C34BC0DADED09CDE7E6090D2D8
:100C50005EDCACD622E0ED2993DA528FEF927294EB
:100C6000A8D29D8522FC84FAF039F913F323F137D9
:100C7000F767ECF6F204AC02F301C5AFBF43C4065C
:100C8000901D05030BB9A9CFD39115E5061050129D
:100C9000DA105416AE205B85CEB83E871BF6F1EC19
:100CA0008A90E3BE228804FAEFFAA5338BB6980641
:100CB000A512E0FEF150C482EE44A8863604B88A3C
:100CC00016600446FE588876AB2ECA66C9EDE12A46
:100CD0003B4D555FE390AF02C258950BD764C2DB22
:100CE0006795AD9FAF5EFF2883F079E5FFA171F6B0
:100CF000EC7880BE5906DB6747805121D34F277BB4
:100D00008B754D97310EF15697D0F55E9F905092AE
:100D100075F26C041363009E7B3D99BED7458D9A96
:100D2000C3CCBCA64EAC9F42D3BC2CBA7996A93496
:100D30008B62C07EC17368C2420C3E0B07CD09EBCB
:100D4000C3350D077769D1E71BD1DDF7DF41D5D674
:100D50004414D567D710A8EA92EC04E23F26199212
:100D600057CAD1865F74D23C038C09D04B90497F1F
:100D700028320D8603263D6AB382F5BE39D4637AE4
:100D80006BC405C70718DCD2491FCBB58910517B4E
:100D9000D7668A9061B3E96A4EB2C4E6A1B909E6A2
:100DA000E4E2CB228CD6E1A1E35A4FD388185972E2
:100DB0002A34A3C7FFB9814783F5455FFBB1894F4B
:100DC0008BD2B48EA290309E725C50969654A85AE4
:100DD000C66444E292A0FFEFA3156D63A732C8D7A3
:100DE0000AAC1C660EB02CB26B0AEE3F7F25B983AD
:100DF000BB99715F773539BB4F0945B34F0628B6AC
:100E0000F113BDB011BEDD01ADEE0248E750D15285
:100E10009358992F934161F76F5D65688941A4D418
:100E20004C4D6DF383B571130FF1213D567898B297
:100E3000F71FB5FA2C88B08EFA0880529A08D1B400
:100E400018BD81C27C41F1BC5E14306AA7B8170698
:100E5000CB591F86B1B8D11C9D27F9A45831CD14A8
:100E600095494FF6091617743D44EB6AE7C409DC4F
:100E70002160EDC24FDA9D123FF425A73BD0B806A2
:100E80003B4101F7CD11D171B228CD26670911027E
:100E900025ECD6FBDBF8801E3B5415CBA5545774CC
:100EA00057AAFC824916C41E8268D3377B4285BC90
:100EB0003A7001A4DF1E0F5E89AEFF0ADC18190E1E
:100EC00057662FD91F4C0130C4040906D9386984EC
:100ED00087087B2D3F2CFE2A0320058B43B45194B9
:100EE00015C3E39273F2CF12FDDA8F1650232A1244
:100EF0002B8DFDFEFF02A72AD2848C960B17059935
:100F000006A8B1E88A3BADBCDF2359258B0D579667
:100F1000FCD03E4BB703AD438B60A16857102F4701
:100F20008BAA208A23673D753D6A6F9E79D0B2CF28
:100F3000A732219C8721D1EC85ACFD5AEDE6E1EA90
:100F4000CF01DD824EE22D94EFBC68FAC6FC17AAF1
:100F500033D1F1F007F1C5FA4B9D25280F40B38F2F
:100F6000F15955566A30017415120D869975690745
:100F7000F3920D97EFFCA2F26A1423EB232661177C
:100F80002F0881A983BF99DE22B6A52B9556277419
:100F900055227350214E41E627A901A8BBA299A969
:100FA0004D54CC3E4910476DB592AA3E04F01ADC70
:100FB000BA1803040FA585464E68DC6ADE64B9C71B
:100FC0006F2203AF5FCC1B7A7A70E936467C6920CA
:100FD000FC9AFBA883BABFB20DAAF97EF1D4ABCCC0
:100FE0008D0EF6ACFC56A79DAB72F3B041A8BFDCEA
:100FF000ADE7DB669146E19FA74AF55B97B8A1A4F0
:10100000A350439EE7B9B54C55E484B25970F12220
:1010100015A4E05E77182F5AD6645DAB1F1569AE34
:10102000650EC520D7C571CCCEA3CDB30B49B9127F
:10103000C332C07EC745017ACE7CBDC37B062FDAA2
:101040000A743D76A210E1DF6B245B6EAA18A9B783
:101050001B745B3817ADF33FF3CACD5E97406F0C3E
:10106000F0622B868FC0D1D4D5D5C6D032CFDF73F6
:10107000ECDA5223EF387CC22B7C8B7EFAB4F80A70
:101080000ECCC330DFD1A9EBD305312E1AA0619F5E
:10109000DB74A590E750B09A135A7D0F035671A7E1
:1010A000EBD5ED070B1641CC22107BDEF928B742B9
:1010B00046FC082847DDF9AA3BCA3DBBFB3871C492
:1010C000B3B1F176169061D793E1ED6ED298719736
:1010D0009B4179AE4E441967DF5C3CA657BDA97BA6
:1010E0004F54E31E12B08977CF95B59773ADB96BA6
:1010F0005F448D060523DB52250AED833F8D498F22
:10110000AFBCA37333A01452BB7589386D4D2577DE
:101110005B6C838FBBEE498B878223D697F1697214
:1011200013A18980C7A8198A3D84C0765F8891B2CF
:10113000337295C675BC4F0C5F14ADD65B4AD502B1
:101140004957E30ABFDC4E5640D0ED58190449DF39
:1011500063128D5B1FC8596C9B145D9F27F9CD12DC
:101160006E2C85D66190ADD26F8627286C1EEB82DF
:1011700025853D805C04897A8D3419845426F924B0
:10118000B33223ACFFA86CD202302D1BAF601CA67B
:10119000D50C44DE61BB29AA9BAA5DD60958380E3E
:1011A00053A215D39388B4F29B4CBBBA7C08172684
:1011B0009954BFFF2538CF8EF4FC6BB66938606E4A
:1011C000F5815BB020E85476ABCD792397497D62F9
:1011D000ABE4405647EE51F3DB94A8A6F9794D52A3
:1011E00066D45D14ACAAAFA29520E11DC2B87456B6
:1011F0004BFDBDE363EE549107001034294C691692
:1012000006A8E700F771810EF10B110535F084BED9
:10121000B500F7B6E7C0248A66002CBA9FDE3636E2
:10122000FB2A31FE9966C7944BC9A98E31C5A5D456
:101230004760ED1D232165A45C3A8BFA31B2F5B00D
:10124000ABC06AC6E672D5C751AC09F4BF8BD57D79
:10125000EB22A3BF5D3E1F6C2630582A825EE5CD8F
:101260006719A34FD3802937CF3121EE0713756556
:1012700077DC4D6E0FB821A4E3AC7D60B4552DA88A
:101280001611BD9EFF28976AF52BADBF33DE7AA7F6
:10129000077A3DA30346127F0786A40197B8D95267
:1012A000B74AFEB87FA6FA0485684556874762DCD0
:1012B000A7EC06B31B9BB866326023617FCE316C0E
:1012C000235169BDB926E6CE03FEC6902436D55912
:1012D000CA6073D7634E11E35F4A15C75B4619B303
:1012E0004FE295C657981F121D47FB8B7F5619FA80
:1012F000FBFCFDFEFF0E5D60E34ADD67A7E6C7EA83
:10130000F75039C27B70B15B5FD87576174457CA06
:101310000B4CCD4E0F70B1F2F374F5767BC8D16EE5
:10132000AF4CD3D004CE267ABB946986CEBA35654D
:101330003773FCF29ECC0416A208AB083794995A76
:10134000DB5C5D9E1F00391C0F444586478849CAF7
:10135000F3B26DBE53774102EF049C7663E0737481
:10136000D1228D732BE8A538896F938897D6A11A5F
:1013700065664707DB7E0ACCC5D5271A317493F61C
:101380009532EBE889E65AB0802EA3852DE4BB891F
:1013900021AA8E24E382B21895B71FDA85BB130CFD
:1013A000CDAADD9689A3D25498EEC9B8D1BF9BA926
:1013B00001800365F1666794C522C320C174D3F62A
:1013C000CD4D01AE912A0B6EDDAD71E77384733A9A
:1013D000BBBAD07A3921CFB8BFB41F90BF109FF6E7
:1013E00001F3DD11F5F6692E63E89FE97FC44764D8
:1013F0005DFAAB8EC71BBF3EB5EF636C8434B7E9B3
:101400006D16813D43975996C0B203CD29CB032079
:10141000844A4260815E9F9ED542A162173859126C
:10142000F7FCA678E44E5A087862AE505124E92CB5
:10143000689C5B5E177056E97352D6765D543A0C21
:10144000D0E2E3E0890E3A62464F5B182760B95458
:101450006B4C8E6E4BDBECCE6D54A5ED57B81A5A23
:1014600068375DAF2C40B3597D44B67DEB7E2F0AC3
:1014700043CA6E42C9736178238A0BA0A18ED5CC72
:10148000CC5819954170F741DD4E19054B4CBA2FD8
:1014900087B7412B83747517BFAA6B479DA604B607
:1014A0007778BA7202AC5FFC5D275F5C3936CA326E
:1014B0001560690571A6B1FA6D38D9CC1BB4673ACD
:1014C000B87D65C36B8A2D148B2C337FF5AE45C177
:1014D0000700AB3589900FDAC15339480D026764B4
:1014E000738271624CAC62545DFA85CECB74EAC6ED
:1014F0005596DB8E51F0A79A6573AB76E9B25331FE
:101500008727B754185EE11FB729899A2A851C8658
:101510008AD0998B1D7C65C435A26EAF8FA0C97629
:101520002D6869AAABF4F5D23F54309E7E9C456C81
:101530003D0C86F8999308E62300C13A4154798A14
:1015400021ECC4DEC37F1D65156765414C685C5C9A
:10155000156C5506451AEF496D9873C83F541CC663
:10156000D1508B722553BB6D75523745B55BA56F56
:101570003532BBC2650E676C6D1C3FDE4986B3CC4D
:10158000ADB941F246BC57C82F32932A8DF601A659
:1015900065E454B29118688E8502A339C9D047E436
:1015A0000DAAFBB294DEFBCE6F68DBC87CD6C1739C
:1015B000975A13D607AE2F5AFFDA1956D907B736FE
:1015C00097B2AA3213AE963CAB3A49EAA94B330E16
:1015D0000F08093411104F04DF42D9404A44BF8A32
:1015E000C5F0DE849F1E011C992315EF531A9EB18E
:1015F0009EB8F3B240B018AE0E14ABA75B5405AA68
:101600002AB0D50FB3C8E11BAFCCE507ABC0E943A7
:10161000BD05B942FDF331992E342E7E069448B6AD
:10162000C5B4852214218DDCC37A4598D788354905
:10163000351D81663EFC99B262F89DB6E975E5BA42
:101640001081E10DE11E216A48E429CA35F865F8E8
:10165000D6F41C7259F85D334FA2831AAE44CF0CF6
:101660008D9DD3345316B734CF6E83E9F13E229467
:101670001D0C9346D1E6F12C733E2EE04168EF2C11
:101680000DCA8DD561B6E17CAB3AB3E6396823313A
:10169000FD5ABB7EA66C4FD2854A9D5F27743D11D3
:1016A000F71C867A7B646566D384A5C6CFC4EFA198
:1016B0009D60E955CFF84A8F831985FE91B8F1AA4C
:1016C0003DE76D98B9308772334C9666D995F534FD
:1016D00075A0D3EECF907D5A83D8879A85AF958831
:1016E000C494D18C54CCAB8E35FAE91619A413D915
:1016F00035AC9B101FC61DD2BFEC94A249A0E1BA25
:101700002331A140E1B75F7D82B0A8CA8BC89F7228
:10171000331A148C43423A8081B58188BCC6BEAF6F
:101720008F1434826C80B4962A988092C7BCC0A073
:101730004BED99D096F64FF21DBA90F159B109B41C
:101740005CA290FC8EF4BF31FAF0095487043B5838
:1017500048FEB58FFBC8194A5B0CD58E9FD1B5509A
:10176000EE54142E22C89F192630E4AECAA45F5C42
:10177000A23C8341C25CA7A4125C142289F07CCAFB
:10178000F2CCA00E3A34C4D2F2D44DC86953D4DAA4
:10179000D5A2F313A7DD194CFCC5E51303ADE9D7BA
:1017A00013421E966E06FCF20E688FF5761C579556
:1017B0000B14200C16649D20E672A72EEE70B08AE2
:1017C0007B0169378F9D91F3EFAD959B6FA199E3F5
:1017D0006389E160C101A1436B7541E8DF1DA9BFC9
:1017E000D7D223AD0EBC4FECEE4CEE73B78D4D143B
:1017F000AC79BD8B4BEE263A2B2F3D48E92FD8AE66
:101800008EA880A2BAB4E10F8FFA3A0A1B0D579E38
:101810009A1E2826AA842462469C0D285F66C99ACF
:10182000C36285BF8B18377A3AA6CD9E4F55811279
:10183000BF8CD50657CDE5BB033D0587E346B137E1
:1018400077F191749610046E5DE1F1AB1725E1B468
:101850007465E5EBFB3C9B55DDD24344EC365E946E
:101860005C5636D591971388685666100D781CC261
:10187000533293BFCD38F1BA0E20CB68A03805D1D2
:1018800025828BE846267F3B21E45832C9664C2DE1
:101890006332E0A21AE0D8E23200AB9E5EE88092AA
:1018A000D2EC8416FAF4086E4AF4D80E1F550D4394
:1018B000FB42A67F1B9E692F773985BF87096D7311
:1018C00017318D9BF3A9912367520C972933949A72
:1018D0006B6250E75C21450F57621CA71983284EA5
:1018E000E55CCCD68A48597A024245D0D1DE4755CC
:1018F000F54121989966E17B13A408448248D29B64
:10190000AF34169FAB1E6939D2B01BEEEE5A7C5E27
:1019100096B8B3FE7A982F0A5B6AC5C061348BCC47
:10192000CDCAEB2CB3D27A0239A83729BF2B4FDCB2
:10193000DB0C2F78B91C85845EE84BF6A700554870
:101940007B46FBC2F85A72A4401E6554917F10FE7C
:10195000270A1B22964C6717ADBF5574C1F44B483C
:10196000CCF5E1FA58C9D1A3CB7F6FD82F21DD3652
:1019700016D8875D89976F32CF93FD705872425B9E
:101980003316171695C85F1C422C0D8CCF36C32614
:1019900061CD31A48086AE3ACD8292909DBF9FF2F8
:1019A000C562986237A637BE74B8028AEBF2D36676
:1019B0006B206D5CA810CFDE21D32FA0829C2886DF
:1019C00057C577A36BA871A465BB6349DBC7D5C9AD
:1019D0001FA5655A12DCE042FD19A5168A4E9052E9
:1019E000581AFEA0E996F717588A0BF375A69F9A26
:1019F000E120F708D49A03FE50E28CBD7BEE0FEC99
:101A0000ED4A4BF249F095A26DEAB49829F6957A21
:101A10009F18818603C2122A41C636AE472EB5886A
:101A20006D5C1D2429273792FD523901618F092AE7
:101A30003DEF1B3820264727CFB2569A2AF461542F
:101A40001D4B0628C93617D51D6A46E67F5038E675
:101A5000783DE176D3979741C3E213C0FB82838040
:101A60001892729424FE5781580AD3309818FD4278
:101A7000A57A9D980926B1B2457FC3404173CF4CEA
:101A8000D79F2F2818EE31F447F4F72D2CFEFC16C3
:101A90009596C78DE1AA1F185D37A91D815EE2DC0E
:101AA0005D831DA0B1EB87147D12B3A8ADD813BC24
:101AB0001B5C9B6A241C829EF0D8E65AD454F9DA47
:101AC000BBB4FDC7B3E6B1B40F803E20C0788F87AA
:101AD0007D86414ECFCBBBBE333419D611B2BF0A7F
:101AE0001E70E3F24D489062955A1D4EEB525752CC
:101AF00046FEFDFEFFD4CDE0392AC0D2A9E68746D6
:101B00002080F0CDA15495095F2F9917D4B65109C3
:101B10005F5895A5530BAD4BE08A6DA254646AA63D
:101B2000B2FB695286F6DF930D7C6D9F93649BD266
:101B3000DE9CC530A72E589E2DB999E812E4B496C4
:101B40009E8C275973998DFC7B49F9F81B07D56941
:101B5000174FF3E05F9D2121EF43E05E7C15555761
:101B60002BEDA9129CB1BD377108245A0B72452C7C
:101B7000B100D79E3BEEF02E6DF529E8DB0D5D67D9
:101B800057D929F213F2C03FCA304456EB96D0B66B
:101B90003536A16743F18D0C0998CF6764BD75A4F4
:101BA000B6000392F7AD1D6A8FE2C52EFB4DA097DC
:101BB000FB7561A295FCEBFEE5C789BD4BA34D49C2
:101BC0002D2AF1983170DC1AC09858005B339DA61D
:101BD0008366800A793883793B91491A2164C696D5
:101BE0004D104B369A5C690E55AC898F23B4A6070D
:101BF0002789516695AF3D7BD7E9D9DE1ED40F36D4
:101C0000EDB5A54F23D9CD6E0FBEE943B35535B021
:101C10005230B3E2B5DC2744AF332F4CE6EB55C06E
:101C2000E1D0C74428CCDF4C4A742948D99278E6E1
:101C300032907119CE8C520C7604080639A6C48EE7
:101C40003766314D733A5B6EBE9453302BD44A5095
:101C5000275621346426115A03784F86E32DBD1F81
:101C6000C750E8BA82AC7F23DFB5B95FABB45E7B07
:101C7000AB14F1E9464C30524248C9A340DD2DC2B5
:101C80000F8D4F06442D4D5F1F351D5F4B8EA52CCC
:101C9000EDC361F6527C687E9F7A99F807E5E97298
:101CA000555D60D6B21C3C8AAFA4C39101B2138CBF
:101CB000CDA3CBB41E48B9A2BA18F96D9EF4C7AF34
:101CC000C9A169731320B953D1E4DB8E776171EA3E
:101CD000D2DA45B8B9576AA7372929232BE521BBA2
:101CE000470AC02E223C382EF5C833675BA955142D
:101CF0001512273819C6BDCBDFBE1F9A0D2EF27AFA
:101D0000E534A37ED72854CEBDE4FB66CFB6E9C246
:101D10007D3AA77D793A2B1E6542639AE1544F358F
:101D200017A79D6BFB3DF9B33170496E46F0F2FE8B
:101D3000B379E933F7958D31328C046A4D74E376CB
:101D4000A51DE1A4146CBFF86FBE697C5D2433B996
:101D50004E80D88293F759549355B91E7B6255A093
:101D6000572611C4658C7B5DB9085FCD4B92B306D5
:101D700071003702159FAB69FF2EED883F260C5688
:101D8000B3BA237E215C0A5B4F889EC73B7EA5B316
:101D90005704485EF5C09DACBE08E9E37B58C90412
:101DA00081D03ED327FC72A713ED19F0CB1E05544A
:101DB000CBF2CD96512BB1DF6F9AC086A778EFB0EA
:101DC00078BCB48EAE90D86AB399950E291150079D
:101DD0009BA4BBE1B7EE5158CDD7BCDA8AEA1C769A
:101DE0005BB23E9367BC32E753792D462638938D1C
:101DF000EE20E052F185DDCBDF182F7A944549AA19
:101E00009230DEC7D34E4B2E2502E900B440D4C633
:101E1000E5842108E3FC977400F08BFDE551F5693A
:101E2000E2F0939447D0B921B7F06C9A0BDEB51766
:101E3000FAD201980386589E3F886EA0CB65894CE4
:101E4000F2E671284943F7EE35DA53457122AA1BB1
:101E5000771ABD7826C448C64065C1806ACC373041
:101E6000C3228B868FC87F128B15E56A956B5B92B8
:101E7000E6D821F4F50A2F2A2D6434A67F6EBEBA67
:101E800087646B68475CB2F47074DCDA26D6A98A82
:101E9000EB64FD987900BD72D5B3F9430354BF5686
:101EA0009DC7F989D3065114B5E2D3C68F7BCF867F
:101EB000ED5C0D00B18E9D123E843B43867169340A
:101EC000D8822D876BB0ADD4C552A970CB12E9DC96
:101ED000D17CC1CB91AE3D7243FE0B9C5DF2978AE3
:101EE0001116171444C0E1824B88AFB0CBC61976E7
:101EF0005B4243401FC9DD40F6D833665B4AF516A6
:101F00005B5C5D72B6CC276D02CCDCCAEB42B21CC6
:101F10000CBA6B9DB953238061C779B64F3479B63B
:101F20007EF06CF22D273373EF5600EE8F2DE13BE0
:101F3000E391E1087CDC149E1698549E6A9431F378
:101F4000977AFA5F978C018F8FF4A816A9D3A1A670
:101F500046F070822731BD215F7299D05B00771601
:101F6000152715726DD230AE52AC0D17AF49A5DAF8
:101F7000811B050809C77D3B5F98A7C02F304056DD
:101F8000D33A9BF079ABEFAD6D8B238D2BCE37938E
:101F900043044442A9AD72B37B797906DA9404769E
:101FA000086571580FECF30B6F82528F6BD054663B
:101FB0008D0BD58363A2901EE1F11DF31FA989C784
:101FC0008B8911CF179BC7EE65A8EC0ABF9901DB7F
:101FD000E76101BC3D4B89DEF5929950DBFED5C728
:101FE00033548C365131245B2FA7A994151765AA59
:101FF000A7AC95A2FDEE9D005038137AB1F42CD217
:10200000454F5CD22D35C927CB755507AFB1C5A358
:10201000C76A2BE1EAFC17E93518939A4FE1F548B6
:10202000C98CC8F64DE35930BDBA299439649B2652
:1020300099B288E203F657347FF199D39F26552849
:10204000A4C9913245E31DD92F0C40F42BA185C6BC
:102050003967BDD0D1EE0BC2FF712B17CB540FA542
:10206000179A34CA1EDC4D84F488030010C824AECD
:1020700096A028DA2A2C31AB5F48B28757E039A204
:10208000B2404C42D23CED785A48893CEB3E65B2B6
:10209000078CE188639637B41F92EECE4270CB8BEB
:1020A00072D42E96F3E0CD476F822A4AABA8E9920C
:1020B000E78161DC23901816CA18EF6594DEF57C81
:1020C0003D0D0FD2DF806DFAAFC2A9602BCEAFE617
:1020D0006D60040AA6A0999E27853D2E263CE03619
:1020E000C1DF51980C3D7D2FB3D5CB8F2F8045FCA0
:1020F000475A017B2761410BB96C0BBC3B54ABB613
:102100009797B51D671EAB4EB1FA49B444841B4086
:1021100027BE1F62BD1C415E25D883302126A7AC97
:10212000772E8F8C3036DA64FF0F50EA9144D1C697
:102130004B043317912505279F34EBB6A44615E8C9
:10214000D7EE1092E90C0C8EF348B54A2524FFCF48
:10215000832E72782346AAC23AC29988A975C564AB
:10216000A51070C2C180B72403DA85B8179877F438
:10217000E7DE01DC607C6ADE616A87681B689FF6C7
:102180003D70ED8033CC931F48A88934CB3A053895
:102190001D3AF842110EB5FDDFB80300810255A0CB
:1021A000B7D7187293B20DF0E6104DCA11845142A0
:1021B00047320B303146DD68BF2C481E3FB4D46631
:1021C000AE10B012372CA78B74F2A93E2FA458067C
:1021D000673486E2C9DCF7C1ADD56BFA9B829FD626
:1021E0009D7091F8697693EDF51F49E08B4E782646
:1021F00087EA01A8039C0F8C85661A00ECB40F4C8B
:10220000B71A0B32296C08CE9ECCAD180AB4B7664B
:1022100066C0A502634ACB821F8DF95ABAF4814980
:102220002AF4554E1306274EA522D50A21C48F89BC
:10223000F2E0010829FCD2439B7CF9CB834235C0F4
:102240004130AD124DBE8DF0B30857D8838B571C6B
:102250002BA4A1BE42CCE45A2E246826C6E00A84F0
:10226000132DB5800A348127D70CE98D22DCC1A15A
:102270009EDCB5704F90F13A3F0FB9D32326E1D1E0
:10228000D5D9292027BB7F89332AF57619363F38DF
:10229000FBBA7682B5A62724C3B8AF46A1D47AACE0
:1022A0005717030809961752E5C48DB8E9D84FD9D6
:1022B000A7ACCB8D899637F1FFFADE70FBF6299734
:1022C000672AB7F2A5372D78AFDA93A679B0D3F0A5
:1022D000B176ABA92983B792DB2C13D5475E891C55
:1022E0008B280DE0A1ACD312F3F4F5F6F7F8F9FA68
:1022F000FBFCFDFEFFA106C105557520C5F0A0B091
:102300000E453502DC312B1017134F9CC300E3023E
:10231000044A116A596686E294CF100CB0065A043A
:1023200082F00020C24A00DE1DE22E0277590555D8
:10233000B5414D4999918A08729584035555654771
:1023400053256A41C99A1076043101C0C0B40F44C4
:10235000F080544599599D88213235880B048203B9
:1023600010D5DE4012150066C43330094019045000
:102370008050508E5024A46A0021208A4001565576
:102380002521218490D1646346A216D8A41060222E
:1023900054423044744A88111514695520B80726F0
:1023A00078100846002C06885C090902000000002D
:1023B000000000000000100300808C083121231071
:1023C000C14110130011D025D8C74431E18CB7A00A
:1023D00061BB987363501021FB4026118520485241
:1023E0009110885801008488023031006288CE3C08
:1023F0000044511444898988B8BBAAAB2B12210030
:102400003233232213757700C0CC444566B9BB45EF
:10241000B4BBB888894030885DF83333D1467844FE
:10242000EC0010519D2ED1552522A200019099D982
:10243000DDFDFFFF03C1088C302148844C0001D32F
:102440004C4802D8940CBEF240B0C43C0C8A3712FF
:102450000E59DF049DF14D100EE4233F001232139C
:102460005011FB0C088CC0400101AC1336C8045954
:102470009D531659DFDF1C76B3CCB8D30E88030109
:102480008410D071A1885335D2ED50F04404C900B6
:10249000D160F3E24E0C4A27032501130973390C6E
:1024A000D8FDDD335D7C13163923CA271010252093
:1024B000560C8C443B5114318413D00E6BBCC78432
:1024C000EC3A120729C400C4332817188010C944F5
:1024D0002D63E022084548D1FC0D3FC8FF480F0C92
:1024E0000C0C0044328C7D1001A124170F481DF202
:1024F000760924B70FAA0A2010AA0A1093402300D5
:1025000011A4884C70CC12A31C0572801DFEC45C03
:10251000DC4518D4F9001B13855B28843F0F0CC6DB
:102520002C41CC473C414C473FA66D4B1B102F49DB
:10253000515A1C17731041C700B0613E1D5A144414
:10254000FC813136463D48C00C51301180C41C0816
:10255000C22183CC0C313311D15060B13E4721846C
:102560000C4C14F1CC0F03CD7004673192BBCB330C
:1025700000282333F100B3C6000448C010222B1FEB
:102580006A33EDC1A8C118033450048282A2A007A7
:1025900010462466369F04351789A0D42C3EFD7E54
:1025A000008F8D7D3113CA30623C4C84E020B654DC
:1025B000F184F640282EED3543150044E2C861143D
:1025C000F111D507D04F4C37200730C9F1BC348BFF
:1025D000D29E615020AC547685D1024BD80D4D046B
:1025E0003348814C11CC481014C15C684C43A14164
:1025F000D98C7B0F0091301A074338404C4F0800AC
:10260000C03040A802C04444C154040133F947110A
:1026100038453188EC041210000000310424044CC9
:102620009381C00C00003002100243147140084C2A
:102630000C02C0880C7037A809002031032C00124E
:10264000302348088423210386101AE28A47C8A849
:1026500000E160A06E08205020C8402420C840003F
:10266000C68C008DC08884204A4C0821820002203C
:10267000444004C4930220A0083258E54110BF74BE
:102680001D48F4841C9C0320A584A0FC3D3008C098
:10269000D280C4F4432C82A812B1110641F4A16384
:1026A0006C72890820134212B00140088042408AAF
:1026B000E4937F24CD03178282C31CF2FB000C1429
:1026C0000C046063180031104814071002044A8A91
:1026D00001D336D8BD138C080182A028CB00100B83
:1026E0002050428155CF838DDDFB33000B000080ED
:1026F0004064F9BE26C107034CD80D01825550D164
:102700004FFC0452F1074515407C0011014442BDC5
:1027100043CB4008820C08820C0832500CE00021A8
:10272000002120412204C4F958D8C4D304118D4D8E
:10273000464CD30E91AA0CA004AE38BF87B807FF51
:10274000378E8B2C71C7D9B80F1447082E8A0720F3
:10275000FF424FED4700360104E38C4310F4760B43
:10276000A2788CB3494800126260173B020018B28D
:1027700048B84354085400E25E19942C719B01033D
:10278000648816638295D54442213503A4041D60F4
:1027900014072029D0D90A803020E2FE42A51888EB
:1027A0000009680A0045A22461C02935728C5F20A7
:1027B00016640F31045DEBEE95F20C3FA73510E285
:1027C0004C431041C8C3BC34D33029F140E6F82350
:1027D000124EC4713D379F2BF77A13AD1BC4103FC7
:1027E000A85606A2FCA090D2C61FEF4F4502005586
:1027F000003108800222840348443230A38BC2A2F5
:102800004B88C0000EB0359381408E4C041601C138
:102810008D6098418E04862806D0C44C040A31236A
:1028200002028130117200098612B3C774C40330EA
:102830009530C021F0123031C12F5E002241B1101D
:102840005402C5805412317280EC9C8328CD04322E
:10285000D2C8C858CA4852858C60858C24858C6043
:10286000C5503212542923622523489532B256218D
:10287000C830A2C4C452100544515511114A5554D0
:10288000554985085E1244554445149415554554E0
:10289000557454D1552195CBC40510C509C13009D3
:1028A000022042204CE18E8EAB4F2010B9E4C6FFCF
:1028B000FF4D1763CA00F2299D30148F5111A036C5
:1028C000120412D0E54948507AE477086109EA44D5
:1028D0000D2060A03E80820A2205143C445F04144F
:1028E000420445421253806541404C4C0462C82169
:1028F00020C4A841F2CF4F723BEA0A47A7290564DA
:102900000F88A80C0FACEA206A5406D8223C573A2C
:10291000271A2D06FF452144435589C68E666776E2
:102920000D7CCD2E2F84DEED4B1732BDDCFA789A6C
:102930005E3C5BB9BB614D7F0F404102C32D497ABC
:102940003E2A2E7E583622624132980C674C3F0157
:102950007D3A92D6622CD83EEF8B7986471B7D91CB
:10296000EA6CAE0E6F4B73920450A5359BB1A56A0D
:10297000658463964CD74B84F69FC0889530C7AA70
:10298000BBD631FE6F70440EF208A6984E38400652
:102990009ADC869A9BE4B806B30C21A2E3C64C36B7
:1029A000C5A04899A36D86B63F1D96FF0B11113F38
:1029B000F5F4B4FEAC84E823B53838C62A65D5A84A
:1029C000D7AE5107C91C96C664006282E04C60D045
:1029D00017A36BA1B9862D098582837F4F5EF521F0
:1029E0008D8A79292363685A4542695415FA25323C
:1029F000C89A31B92B33CD211FD4880CCB371D2178
:102A0000C751065269767774DF538121037D569B47
:102A1000B37A7B7879464744454243EAB07C9E7E50
:102A2000207ACE1E3FF682FE04D7F9ED515EA092C9
:102A30008D8AA1F60C8CCED638DDED5A8FF32FACF3
:102A400008C04ADA2804064614C0169A78738571BD
:102A500007181119B976D7BEB78FE3C0233C3048A9
:102A6000F6428D7285D039F6F63A1310111E818622
:102A7000EF63A9492BA71595D79B918993BB7F59E4
:102A80005B9A5E78E85CF27485E2E310DF1CC5C9EE
:102A9000572FC1BD539FBD270B60D4A0BB4B300245
:102AA000883505C833D6D7D4387812221821117248
:102AB0005870F246F92855DFDC55DB5F6F544A0643
:102AC000AE53599143E17686F8A579CB8544A8D0D9
:102AD00017E3447669BCC2847A4CB99BE171415CCE
:102AE000F72498E823B1F6663C6D5D9091A40CF84C
:102AF00037B9FA6ACE9F5ACE6A272E12A0C4F65E64
:102B000008C0FE0853D9170638D872771DD4566905
:102B10000F97D1097946A08AFF374340414E4F4C69
:102B20004D4A4BE210A42E6E102826AAB290443CC7
:102B30002F27F191F3E7D53560D01252A05CE69EC5
:102B4000C480E8D1DBE39DF14FC44305C3EF4DE5FD
:102B50004F6F3B429B19677678A8C63278BCFEA6B9
:102B6000FE660608096CF87415EDDD6A027E1F49E1
:102B70001DB05A621D9C40847B7873E5579EC2BA93
:102B8000BB8AEBE84387F7A2C3D25155F1FEFFFCA5
:102B9000FD1D35020EA6BDB2B342E3E01194AB6E4B
:102BA00032AA61C13BF9B6D42A1CA93BB174E8250D
:102BB0002F3922271708620EE40C51551BBB059DC7
:102BC000DF8FD1ACAD4C151AF8481192135D97C93F
:102BD000E8AF1E5D5D2293D0F1F4D59627686E2D87
:102BE0009CDBFAFFDE813073773081C2E3E0C18283
:102BF0003374793B8A35147343D145C74BFDA17BB0
:102C00004B0285257E50A1BCDEB8902EDEB4A74FC6
:102C10005AED5D572781A9E38FA91D4767F569EB39
:102C2000679D61A24F65959C1B4575F37771019B6C
:102C300077457DEB7F810D2707C9E97EA77818ECE2
:102C4000ED023DB629F06156CF0C6596516842FF02
:102C5000F331F9824F7031F2B78F0DA2A326F5FA46
:102C6000C3CC1D007320E1A2163AA926A38B35DA46
:102C7000959C330E87BC673E6B61053F27A06F7C38
:102C8000A016AB6D75D62F289DF2FD0A9D75D52334
:102C90003B346CD265BFEF80EFB31B089F55E982D0
:102CA000A5D413B052F01F4A8FE2C51847F6C902E7
:102CB000B584F1F154CEF2CC6DDFF86A7E88776D81
:102CC00085226AC24C9CA6D36FDA9DF769D6C2D41E
:102CD00075659D202A7C60E0AD0A32EA34A42EA9F5
:102CE000EBECEDEEEFF04D7A171C2D8E8B500502BC
:102CF000BFBCB10A8BDC49A7353937BE91993A8DF3
:102D00003F912BD2ACCBB5CFB6A784AF85918AC704
:102D10000F8D08BEE43A69111547146C31BD1A9F36
:102D20001FA00BFB8CE695E59697A481A583AA8F3F
:102D3000AF07A8E6C4C341A042AE476644F39AF683
:102D40009FF698D66E21602563DD1568672C684A6A
:102D5000695A14E0A0A36184628F674C6476BA84D8
:102D6000BF93B883689F79837AFE35443378597C62
:102D70006BF934CE33F7982EDB88AEA73BC679C407
:102D8000FB146DD6963473192809550C271D39D7B5
:102D90000B1AD4467FA0E9EB95919095E3838CB113
:102DA0009FA48DA5E6B090B2E1B4D7F1C2FACD8868
:102DB0008BEFFEE6FC80D7FAE54BE670E420CD3ED3
:102DC000CE33CBC2C8DED9C2DA93C3BFC1D3C9D018
:102DD000FBBAD9D0DAEDE78EA393D59DC768F98108
:102DE000AB99DD94CF8EE13E2B2E3736143325215F
:102DF0003818F12F7F59A50E22B9248A7A82FC1A3D
:102E00008A30FDC383B1992B9B186C99725C38B6DC
:102E10000E2EE80E7E6044AA536965431B4B27D9EA
:102E2000AAA0CE00214ACF797BF806FA14FCB17E25
:102E3000679A3BD8565707C58D8A661A25A6060697
:102E40004C2DED40E9FEEA1EF26B586AD6D41FC93C
:102E500035920104014687215DB031B589897FB281
:102E60002552A305C1A8536CABDADBC89C6657D4C6
:102E7000F5B2EEA64158EF6C57D036685EB4E75213
:102E8000CD10F09A6183BFF0601AD76C64443AD6D3
:102E900020E5DDE7DFD9E1032B21E5EF9F79E58B25
:102EA00097B20BA849E5A7DFA568D3E25CE64482A8
:102EB00077870300AE60CC824FEFD466CA88854D19
:102EC000ADAACDDF6F5DED5EEC9A89B08755E196D6
:102ED000C062C33E31AE8FBCB78B710133F7BDAD5D
:102EE000FFB3713E73102D6263E465A667E8A9CA5B
:102EF000EDA01D6E6BF36A1EFA1099565B1895EAE9
:102F000057F519925FCCF14EEA0049F60BE10D0638
:102F1000FBD45505119ADF61AB683EEA346077C493
:102F2000E576DB3D55CA7DC5BF1F9B38F9F6776650
:102F30002B6CD354C56F2B5969CAAB1EA9A6A784A5
:102F4000A5B6D2C0B47EBF34881ABBCEB91442D461
:102F500095B2D305718EF98C2F6F83918983A53536
:102F6000A3205A261C11D1D1373FB13ADCF462FEBE
:102F700068F47E10F180000EB8A273A1093BA7ECA3
:102F80008B71B5C2D0087FF49311A987370DA14288
:102F90003592BBA5F14E9A76F70B8345C9E6D4BEB0
:102FA00045BF93205C9E657C5DE0166E3936F7E682
:102FB000EB64212E2F9B4B487D2FDB1E6986E71289
:102FC00045D2AF65612A7F28A0AAB3C859434116EC
:102FD0006C107ED3E36BBF3A4D7C4B2AF824F66C21
:102FE00085369E362ECCBDB98AB408723BC7F4C66E
:102FF000B75C431E4F58478E2238890B3AA981236C
:1030000033C0AC8783E1DCB39B71295AB7A6E8D5FE
:103010005540672811AE6D82502C2482AB1BDCB664
:103020003EE096C8C8B4DF89AFD616F7FBA3D89A9E
:103030002582ED629D4604167E089870F6E048EE03
:103040004349D1C250D8D5479FCF7D53FF1629623F
:10305000EAF40304A923E96435D803D0A98664CE31
:103060006D147184241A3E6EE3F8624061B957838F
:10307000E7F084E329D8741E85D2F5BE9992673CA7
:1030800097AF5152F32672847DE85F5C1BDB4D0DD8
:103090004740E15455CEAF4CADD8B92ABCB4D54465
:1030A000686E796C014CAD585D7AC918ABE31F149A
:1030B000B5CC85C233D3BD28335CA35956044D83A8
:1030C000D540A6234F6971B235F789C399A4DFEAC9
:1030D000D340BFC997AED7F10D46168F4350470A6C
:1030E00021E6E724051ABB7EC0FAF3F8B118B33025
:1030F00011131DFEFF505C727E94983B391627C257
:103100000A9E45FB01414F636D858B5B5985876343
:10311000D79056A6F91387648B818DA72585879B49
:10312000832D89CF8F2E8FE26F96D35552F4B51928
:10313000561C16B65260C544CFA54603137505AAA2
:103140002E80415BEF5E89FCDFE956DA0247E8F248
:103150003BD8195811107D341A47559C05776FF5E7
:103160005BC46BD10DBB41C2B5626966F9B293C64F
:103170004B7A474EF395AE8EB05C09FF0850C7BA44
:103180001D30FDC09380972EE35AF7748CA0972AC8
:103190003B7C1143B046473F99A4C7B9A5E3999A30
:1031A000AD9721AB8580017983E4B39DFF7B31AC82
:1031B0008BB621BC98F07389F3B4C3F5B180F9667E
:1031C000D0D0AF1581CC01C2D568E540D144DBC970
:1031D000538ABEA8642959D2D3F8EFD9F10AEBF982
:1031E0006FDC2FED99BBAD90913CB680ACE45BCA2F
:1031F000BBFAEAB6CFD85A742034DF2D713339E8E0
:103200004395B554519607941552530A071E958B52
:1032100030A02D18513C316413BF9956698E9544E6
:103220005B9C618E6B158B7C2F2437E6A73E850A4D
:10323000619C0092833012D6BAC5B565BE58E78648
:10324000EB3C74F683A5CD5972ECFB37C979E103E9
:10325000FF24B3082F8E684602F8EE6F43C6046859
:10326000A3F52DA2B8153582C3DFBDD8CE38D2B2B2
:103270002E44F6D0B7E1BDE133353DC0942EC7BA38
:1032800082F525B513DE33BA963CDBE6AF14CA06E9
:10329000B9BEAE0713F42C75FB04155CC446F00EE2
:1032A00051971C16C11E000A0A1C5E3AE488B72614
:1032B000D9232432EBC7B86E4DA1E128FBCEACEE8A
:1032C0003E64232E36C098762FC8DFEABD12CF5B4E
:1032D00017BC83A22540C7BE018419A007D9F59A5F
:1032E000A7C72046E7E35973F1C5E958F748B54148
:1032F000FFF9555DCE1C4D210F7326B63BEEFC96B3
:10330000301C2E5E1C809D3DB14C801411F599BC83
:103310000744BBA7BFDE6EC4387875FABF74722449
:1033200065F04D7EBF762E28242EFB2C4C219D86E9
:10333000A79E41965CB9510CDFE6794D09D4EB4468
:10334000579CF17E154C81EE23E468FAF9261DDEC8
:103350009FA242D6975ECF1C9D7B2DAE5988E0423E
:103360002747CB03C30B29D4A6B47B4A4408A18AC0
:10337000A35AD7ADCF609D20028727954F04221313
:10338000071812372F9E6F4D753FDB4A0708C93C5F
:10339000DD8B875FB1C0FDA0B8D26B685DAAD53662
:1033A000A90F25E8F1CCF7F94F12F39D4B1EFF9DB5
:1033B000BD2193A2BDAD61C36740810ACAE7A7C61C
:1033C000BCC0AAC6521C191E62F79C9AFEFA6186FE
:1033D00039F3413C725E7DF7ADC259D631F3575493
:1033E000EDDCBDF2E5BFC1C2B988E92627A353E6EB
:1033F000EB6CEB1CE8625D7E65EFDD82DF0E19167B
:10340000A10E7E9EB30C01A4088406C6878878347A
:1034100011E04764637CC305F37836BA9187399C21
:10342000549A52C8C9861A222FA40E6661E322AAB2
:1034300028ECC622EF90A75473E4438981AE3F1E67
:1034400050106EB2D380DD4D0347C5BCFD447B11E7
:103450008B40F7BEB93CB1C101C2DBD55D2E9844AB
:10346000EFCC235E264677811379D190BC96D77432
:10347000C78633A2EF9A6F98FDBB9F7C7D9273390C
:103480009136BD7153006F948FE4EB08AFE4AF85C4
:1034900021CBA1204C068BD505A2DED83916151CF0
:1034A00061C69A9888ECA8FCC5B511101A24BC26F0
:1034B000BDC5198F1B4CC8E9CF83C9F17F969362B4
:1034C000856A25D7F948CA62AF5249D0E7C8A9BA78
:1034D000EBD4BFB1A79CEDC9E5D4E0A0DBD829D9D6
:1034E0008994D18C1C96EDA41594C316AB2829039E
:1034F000D5FCFDFEFF300B0463CD23130976F7875F
:10350000DC7003EF2529DD74231213B3BF56694124
:103510002B154C32195C848A133455680F4081B9DD
:10352000D2ACE0864EAC39138FA77B462E9C2992F5
:1035300073A93FC7BF8DE94A62F84BF6DE6EB05AF9
:10354000EB35E9B413000182438405C6C7C8097985
:1035500021A627824C5A039137DF0C2E5D50D342AF
:10356000D1220B9356138862D30DD1DD8EF88F498B
:103570005D5BA784983AF826397435EDC2360103AD
:10358000A3C07C4586C6083E0A380C3A7461895B44
:103590005727648E8E004F98E5DF5CB6ABEBB01614
:1035A000F38D11365FDD154ADEB6501A54E65972B6
:1035B000F3BDEDF2884CF2C3630F49A699CD8DB3EC
:1035C0008B807E2F8331911EB4E1ED788F68C742E6
:1035D00065C2733E7E6898A2EED888A62BF7DCD031
:1035E0000AA0A6EF4F05B18BB344F456E6C060C6FF
:1035F00096BC48B4FE508D620D58A74C2846733CCB
:103600005002F04E116951A24D15B5EF574D25AF3F
:10361000534D2F1F4FAC41EF1B5D6517AF51697FB5
:10362000179C732B6F8579F92A98C434369CDF4D2B
:103630008A94309A7B4CDE4ED43D89C2F48462CBAE
:103640004BC066202A9C3F377150D1979BBE6EB409
:103650008C58E05CA957D0F462C069316BA761EE69
:103660008DDD4EAB7185EDF63831C996322C3F6653
:103670006B1A86726A211480B6D60DFB2B5909A2EB
:1036800085C0AE4F238B583E7A58B8D6CE3CA15752
:10369000A3D0BE2333BB640E4A6890E6FE0CE5B5AA
:1036A000E35FA31E2A88587E0A1880F6B9DA50769E
:1036B000761090FE6A5C30C0BE68F46A06646730BB
:1036C000ECD0D880B2EC3C7AE2781C7A79A5E5B7E8
:1036D000D9A1719A124CCF184D61A59FA7A4CEC74E
:1036E000ABF728AE5EBC2CB232B854BABBDFD1B255
:1036F000D81155C6247DADDBA3390B7BAB01058901
:1037000076A0C4A2E1D1BDE7BBFA3E1AD050AA967A
:10371000C4541BAE62803D4078CEF9C5AB376D898D
:103720002783A68C3BCFE5157F234BE2E3B693D4EA
:1037300007E0F78291AE1D5CE31EEA48E9263AC62F
:1037400050408AB4EE52D87A9F859EE813A8EA18B2
:103750003CFAA7BD79F33D88EDD4C5FAA228EF6CF9
:1037600077BA46E4ECFA77DC8FDA536A2957DF94AC
:10377000F1A7DB101AC4D5EF811F1924252A5A0E90
:10378000C3005A072FD4BFCEB196094ED1E861309D
:103790003D743B3447CAA9F8ACA0CF555DBB477612
:1037A0007B42931DA3179FA9BDDFACFCB2FE4CF07A
:1037B000B51DF53A0F4DF9938D3985E5C9760E871C
:1037C0008B078392A980420F935F08568AF015A752
:1037D00018F70C5EB986CF98BBA2DBB83FEEB7F9FD
:1037E00075E23532337EE2DC9107A13D6F56A104CC
:1037F000E09A3350A34AD6ECAD580BE06C3252CC71
:103800002D2ED360F5705F0CF3D2D65B57B877518D
:10381000592B7BF4FC2E3082CD94A81E8228EA24FA
:103820008E2CA8163E90A2BA2E70B97DAFEC7369AB
:10383000B214F1A3F86EBBEC0D9C0B1A17A6E7921D
:10384000E5F7B7F5266CE23313F718163485D90778
:103850007390FC9D711A39245D9EC458BF2E377930
:10386000F5B433C0015E5AAA9D12AD2A396B5BF4E0
:10387000885293AAAB532F1A8ABAD8BEC28A7CC286
:10388000C5D42CC6610B401266D4ADF0F198DA5B5A
:10389000DBC73CDEDC8921818D5E0BD88434BCE43F
:1038A000B5926340BE8EDF5C5DBA5BECB95E92148C
:1038B00001B25350F15C83D56D4A8BA81B980781E8
:1038C000E9023E802144260619171D9E7278A4C085
:1038D0001394157B7F59F7474391F34347CDFF621C
:1038E000E24AAFCDFFE3A1CEED0C092E73FC21C659
:1038F0009BE2156BFD6545F28FA41CA25B8C993190
:103900002576084E6A54E1E94F4410562C1637606C
:10391000F8315D506F58891A4BEA9B380FD093B637
:10392000C1C6C794C79ABBB8B9DFC4767948D7E295
:10393000C326A78485FA5DA8A5AC7DA83F60F122C7
:10394000F10A71B097BE0DB26350C92527685C4675
:1039500010FDD54526205164FF145D88BF90BDA49D
:103960007F8793C0B77BB0DE6E4C0C3646D4C4D68E
:10397000A0B5D1D0BE2CA0BAFAC4482A293125E975
:10398000422090B6F6D05C3E3D513913AF45D9D1B7
:10399000D6DC76D0BCBEEF1CFFF4467B27F58166F3
:1039A000826F3E732FED997EFE77FE08E0D9F9F124
:1039B000B5C4130091BA9984FD9A1DDA13BEFF9E17
:1039C000282223A517BE3F99F5530DB8F1077702BA
:1039D000D5FF0570F4384F3A8D7ABBBD69F6CFD16B
:1039E00033103580499ED7B9953A4BE8232C3AB429
:1039F000556413D0897677747504E43C29F2A7AA3C
:103A0000D7C2D560C1E67134F52F73F809CC57D50C
:103A10007DFCBB5DBE1EDFCDD5FB2BA83BC6A376D0
:103A200061A34B283406D17C11FA0BD8F523931CE3
:103A300035FE1ED011BB9F71C92A6368BC222B21A1
:103A40003517A3C8150E7B1CE9B41816DA64A34D0C
:103A500015FC01A874E6977DE5849379295B230022
:103A60003DE4B9BA8FCE1FFC2BFA3B51EF76995C3F
:103A7000B0201F10BEBEAF782D0081D894809790E3
:103A8000E5426BFD41CEEE4E4700ECD1B14344D24E
:103A9000583DD5C2ACCEC70C909E2B558946CFF968
:103AA000374E86CC4DFF93EEF01A4F1855D3F7E6FC
:103AB000D1B2A1EEB3D367ACCD88FEBF874D896B81
:103AC0004340D670D1B5EFF05D27FB829036BF0E34
:103AD00035B99B3093CBA8AA4D8A39767B124236F2
:103AE00009C78F60B713D77C8D57B3CA9596F7F681
:103AF000F6C1C690A55E0F0EC241497F46714919B5
:103B0000A572FE207188C24A9DFAFBF81976D7F497
:103B10003C84B3FE79EBAFFA05951B28C974B9FA5A
:103B20003BBC7D3E7F2061A26364253D796CAE4045
:103B30002B06E9E16B77553DD7FB11A1DB981521E9
:103B4000DB1C9D1E5F8001424304C50AB9B8890A87
:103B50004B0C8D0E4F7071B2B3F8F67AB7B8797A14
:103B60003BBC5D06B34B2DA2A3A46566A728259197
:103B700027ACAD4E4E9C32B2B01816A87D26F0CAC6
:103B80000F5D0DD034962B64A035AB707CFE77C0F2
:103B9000447AD220815E5FBC5DB72DFF03F61CE244
:103BA000EEAE835401F86BCD6EF44F452F4666940C
:103BB000DE8293441184C5FCBD43DB1CAC6ECF2C6C
:103BC000B08AD668C7DE8F888F5EB7F45980528678
:103BD00015BE7390EEAEA3C5850A063E26D4629349
:103BE000AB47A9EAD15EFFD41547ABA1593DBDA6AD
:103BF000B55AF390C408CA56F4D03B20DC738774DE
:103C0000F89423B0342E7FFCC7808EB899F2F3F07D
:103C1000B580CD98D9FB7DACCDF96DAF6BD2CAFE26
:103C20009002B1AC01BEAC7A3F035BB8591657267F
:103C3000B270C705B19BAF91CD671BA9211645BFD7
:103C400052B17502EF8D11C76BCCAB4311FEB7813A
:103C5000D515153003434F00902643BA87362EF30F
:103C600055A1C136298A4044FE4AF036941939B12B
:103C70001D1A213C587A27612D640126838C4D2A18
:103C80009058EB1A64F0FF7431C282203184090A23
:103C90000B8C0D2231BCF4F6EF8DA62A88A4C997AF
:103CA000E7E2DDCEC1984982E2125DD6B7A4FFAA51
:103CB000DD93757258538F6A1F5455DAD7D819DAC5
:103CC0005BA45850071C26E2D71C19B03C38457835
:103CD000D99EEDD69D3C2DC57A4CC67F4F5E5F5C6C
:103CE0005D75EB97AF957DDBCBEA6CCA2ABA721F84
:103CF000283A08FEFFEE4AF440A23501810E1A82EE
:103D0000D2AEFBF1B6B01FA2DDEA3A58989D5F54DF
:103D10002C40573C29C0C77945C26668C7CE0A4CBB
:103D2000CDABD8E22180CC724A744C761E00776A03
:103D3000AB1AB00646000F1E651415430799155AB5
:103D40001B6D710069804182434450163A18880601
:103D50000B8C7C621146F132B334353327092924A8
:103D600037BCE0560E303FCCAB3A656667594534F8
:103D70006B1A783F12C060CECDE25DC8D7D899DA11
:103D80005B9CDD5E5F0081429ED4F4D6665494DA7B
:103D90003A14FCDED11EC7EFE221E5A7EFE191CB9B
:103DA000EBBDE9D7EF457D9C49BACCF66DE309BF81
:103DB000FB5DF11F37458159A284A0F8D3F7451F59
:103DC000F9ACC1191380CDB0E080F20AA90B95E1DE
:103DD000A5EB7F0A9BCB5FE0B7D35507DDEE75A05F
:103DE000DCE815E44EF2ADB8D468F7E57D75C304A0
:103DF000D4E1B9B05FA13F17A3D585EF5751ADE32B
:103E00005B31A1BE13526EEB53EA4A7E19A831967C
:103E100054E55DE0345809924B7D817AC9377901C8
:103E2000657C052057CD714B734C609259A31740A8
:103E3000427C553087BD013ACFC1790F7FBE7E09E4
:103E4000060C28720A520D961B4711D237CD011469
:103E50002BBC818EF1487F3D1D37695DFB8A76BAA8
:103E600078BC33C6537E473DF6C8A36D2BE8453476
:103E7000C3404B21FA3C57991F94F96869C631B683
:103E8000BDC30832598B8D82AFDA2DEAA1D71C262B
:103E90004D87018E63EE191E95F3201A71BB3956BA
:103EA0004542E3003EE8BF0ACF82EA330B6EA2E64A
:103EB0002B005350F1787DF48C417910DC945976C5
:103EC0008574F1F890556D04C848C5EA3936976293
:103ED000A7EA825B6336FABEF3980B08A95015DC9B
:103EE00094F00FCD9E4CEA774F22EE6AE704B75468
:103EF00086A471DDB3FD5AFAFD474B360FA0390693
:103F000030423D02A720197AB32C0B6810668664F4
:103F1000DC627A60CC7C038D9B58CBC82953515608
:103F2000659491C0C17E4D294B487B582A6274E646
:103F300035C0A13C47CC620E540AE7D1E547EB15EA
:103F4000E933EFB9ED0FF32DF1A3F7112C2417E2AC
:103F500027B2B31031D81D8C8D2ADDDA29AB152498
:103F6000D3D08380211EC94E3D170998993617C2B8
:103F70000732C5C2311C317CA09419C4FFF8E1E4BA
:103F800002D40195C3EF69C8D5988E8AC76667A128
:103F9000878C638583B0FF7E2FB7F523FF5055F0E4
:103FA000ED528EF2FFEEAD7EA8968E16239B59A69B
:103FB000EB5CCCE687CE4F9E9398A789BF74114ED9
:103FC000CF1471A62FF05DEDCA708934C4E87983EF
:103FD0007DD2A5AEB7CBEF5A934C69CD2B48A10A41
:103FE000A78C25228F78B8BC53E8E56AA7D8EA8267
:103FF00015945578C24C4F5E936AFACAEC38D30CCC
:1040000051B03D082F2C47749C7A73263F1E1654DE
:1040100075004D4E117575B721426B8601488FC9E9
:10402000171D733B8F8019F6777569E33B96C9A21C
:1040300055839D222F4667A4735C39FC1B8462283C
:10404000296E6F7E094377682983D31008101806FC
:10405000EB9213646F93C7AE4078F5760937BC6670
:1040600065F40341A35FB9793DF73B064F08371468
:1040700013D4B1DEFB0183CCA5A2499DA1AEB599B5
:10408000C5D07D9BC130449E63644D4E4F4041423C
:1040900075F2489251EEF6FA27EA95A16B8B219AB8
:1040A000B1DC4396E11E3D95FFCB9B186F48F7822C
:1040B000634CD38EA6A6B646F3EE89D141CE51CC41
:1040C00093FCD5B5FF301DC9E314B355E7C8BFFD58
:1040D000EB3CDBB03186B7B16DE46E8807B0A79AD0
:1040E0009344A39ED79869DA13BA4BD0D120B72650
:1040F000ABAC6DA21F53554E4D4F4E5455455745D1
:1041000044544855465249534154004A414E46454D
:10411000424D41524150524D41594A554E4A554CDB
:104120004155475345504F43544E4F564449430021
:10413000000302050003050104060204E240A0C8D2
:10414000A22C2E2FF800238128AC00A6AFA5A4072F
:10415000000A000F0016001D0024002B002E003363
:104160000038003F00450047004D004F0056005DFD
:104170000064006B0072007900800087008E00955B
:10418000009C009E00A000A700AE00B500BC00C3CC
:1041900000CA00D100D800DF00E600ED00F400FB0B
:1041A00000010108010F0116011F0126012D013434
:1041B000013B01420149014F0156015D0166016D5C
:1041C0000173017A017F0187018C01930197019F9F
:1041D00001A601AD01B401BC01C301C801CE01D5E6
:1041E00001D901DF01E701EB01F201F901FF01074C
:1041F000020B0212021902200226022B02300237A1
:10420000023D024B0209FF0FFF0101173B3B630C0C
:104210001FFFFFFFFFFF0001000A00000000001564
:10422000010101010101014F46464F4E2032344841
:10423000313248005645523A20302E383520005051
:10424000582D313543002B202D20544F20534554F9
:104250002C204F4E20544F2045584954005553456B
:10426000204B455953202F202A20544F2053454C92
:104270004543540053455454494E475300424B4C18
:1042800054424B544D434F4E54534C505442454569
:104290005031323234485220204D494E205345434C
:1042A00020595220204D4F4E204441592052554E06
:1042B000434B45594344424F55444953435353504C
:1042C00043202020204241544C42415454001124A8
:1042D0001FBECFEFD8E0DEBFCDBF11E0A0E0B1E060
:1042E000E2E7FFE602C005900D92A03EB107D9F7C4
:1042F00027E0A0EEB1E001C01D92A336B207E1F7BE
:104300000E9478350C945F370C94000081E0809314
:10431000A00480934F028093310284E18093A10432
:1043200008951092A00410924F0208958091A00465
:1043300091E089278093A0048091DD0182608093C1
:10434000DD01089580911C02811103C08DEE91E082
:10435000089584E497E008959C014B9710F0255A46
:104360003109E7E4F7E087E0829FD001839FB00D39
:104370001124A955BB4F45E557E0818190E1899F04
:10438000900111248081822B8D9332964E175F0706
:10439000A1F70895AC01FB018EE0815008F4089567
:1043A000282F30E0DF01A20FB31F9C91240F351F8F
:1043B000D9019C93F2CFE2E3F2E0808191812281E6
:1043C0003381318320832481358133832283268185
:1043D00037813583248317821682089508950E94B9
:1043E000DB219093A6048093A50408950C94DB210F
:1043F0000E94DB219C01E7E4F7E0832F82958F7018
:104400008683832F8F708583C90134E096958795C5
:104410003A95E1F78F7084832F7023830895E7E442
:10442000F7E0868190E0982F88279295907F2581EC
:10443000922B2381822B248140E1249F900111241F
:10444000822B932B9093A6048093A504089567E490
:1044500077E085E597E00C94CA2165E577E087E48D
:1044600097E00C94CA2167E477E08DE192E00C9428
:10447000CA216DE172E087E497E00C94CA21E7E479
:10448000F7E02281818130E1839FC0011124922BCA
:104490002081822B93709093490280934802089563
:1044A000E7E4F7E0818120E1829FC00111242081AF
:1044B000822B9093E9018093E801089520914802AE
:1044C00030914902207F82958F70A901482BCA0143
:1044D00090934902809348029C018B31910538F0FA
:1044E000205C31092034310530F40C94AC212F7E4E
:1044F00028303105D1F70895809148029091490202
:104500009C012F7E2830310511F00C94AC210895C8
:1045100010923D02089580912F02909130028827D9
:104520009093300280932F02089580912F029091F2
:1045300030028827E7E4F7E020812F70822B218169
:1045400040E1249F900111243327822B932B9093D9
:10455000300280932F02089580912F0290913002B3
:10456000E7E4F7E0282F2F70208324E096958795C5
:104570002A95E1F78F708183089520912F02309161
:104580003002E7E4F7E040814F70C901807F842B5F
:104590002F702083218140E1249F90011124332733
:1045A000AC014F70242B352B3093300220932F0217
:1045B00024E0969587952A95E1F78F708183089579
:1045C0008091E70180932F0208950E94A221FC01AF
:1045D0008081815080830E94A221FC0180818E30E5
:1045E00010F08DE0808308950E94A221FC0180815B
:1045F0008F5F80830E94A221FC0180818E3008F0B1
:104600001082089510921C02089581E080931C028C
:1046100008959091ED0180914407981303C081E0C3
:1046200080933D020895CF93C82F0E94A221DC0100
:10463000EC918FEF8E0F8C93F0E0E95BF84FC29511
:10464000CF70C0830E94A221FC0180818E3010F0C7
:104650008DE08083CF9108950E94A221DC01EC912E
:10466000F0E0E95BF84F808180932B020E94A22149
:10467000DC01EC91ED3019F410922C020895F0E079
:10468000E95BF84F818180932C0208950E94A2215A
:10469000DC01EC91F0E0E95BF84F80912B02808324
:1046A0000E94A221DC01EC91ED3031F0F0E0E95BF9
:1046B000F84F80912C0281830895CF93C0912B02F3
:1046C0000E94A221DC01EC91F0E0E95BF84F8081CF
:1046D00080932B020E94A221DC01EC91F0E0E95BC7
:1046E000F84FC0830E94A221DC01EC91ED3021F44F
:1046F00010922C02CF910895C0912C02F0E0E95B5A
:10470000F84F818180932C020E94A221DC01EC9160
:10471000F0E0E95BF84FC183EDCF80911B028093FD
:10472000A504089580911B02E7E4F7E0982F929585
:104730009F7094838F708383089580E180934607F0
:1047400008958AE0809346070895E7E4F7E08681BC
:1047500090E0982F88279295907F2581922B238136
:10476000822B248140E1249F90011124822B932BE2
:104770009093EB018093EA0182E090E090934C02E9
:1047800080934B0208959C01E7E4F7E0328334E024
:10479000969587953A95E1F78F7081832F702083E6
:1047A00010924C0210924B02089583E090E0909397
:1047B0004C0280934B020895CF93DF93CDB7DEB7C1
:1047C0002E970FB6F894DEBF0FBECDBF82958F70C7
:1047D000E82FF0E0EB51FB4FE491DE0111969E01D2
:1047E000215F3F4FBD0181E08E0F0E2E000CFF0BAD
:1047F000E95BF84F90819D93E0E08E300CF4E82F58
:10480000A217B30781F787E497E00E94CA212E968A
:104810000FB6F894DEBF0FBECDBFDF91CF910895E4
:104820008091DE01883620F081E080933D0208957A
:1048300010923D02089580911A02811106C00E94D3
:10484000DB219093A6048093A504089580912F0204
:10485000909130029C0122279091E701292B3093FF
:10486000300220932F028093E701811102C0459806
:104870000895459A0895CF93DF93E7E4F7E0A4E322
:10488000B7E081919D91EF0121978923888387E08B
:10489000E535F807B1F780911A02882351F080912D
:1048A0002E028D3031F48091470780935407809316
:1048B0004107DF91CF9108951092A6041092A504AC
:1048C0008091A004882361F080914F02811112C071
:1048D00081E08093E1018091F4018093A404089524
:1048E0001092420781E080933D0210924F0282E0D5
:1048F0008093E1010895089508950895CF938295D6
:104900008F70E82FF0E0EB51FB4FC4910E94A22181
:10491000FC01C083CF91089582958F70E82FF0E05D
:10492000EB51FB4FE49121E030E002C0220F331F36
:10493000EA95E2F780912F0290913002822B932B1F
:104940009093300280932F020895CF93C82F0E9436
:10495000A221DC01C295CF70EC2FF0E0EB51FB4FB0
:10496000E4919C910E2E000CFF0B81E09E171F0618
:1049700009F080E080933D02CF91089582958F7079
:10498000E82FF0E0EB51FB4FE49181E090E002C0B2
:10499000880F991FEA95E2F78095909520912F0254
:1049A00030913002822393239093300280932F0220
:1049B000089582958F70E82FF0E0EB51FB4FE49162
:1049C00081E090E002C0880F991FEA95E2F72091FC
:1049D0002F02309130028223932321E0892B09F4A6
:1049E00020E020933D02089580912F028093E701FB
:1049F000811102C045980895459A089580911A0240
:104A0000882331F00E94DB219093A6048093A504B3
:104A10000895E7E4F7E0868190E0982F8827929543
:104A2000907F2581922B2381822B248140E1249F3A
:104A300090011124822B932BE2E3F2E02481358153
:104A400037832683228133813583248320813181FA
:104A500033832283918380830895CF93DF93E7E4A8
:104A6000F7E0A4E3B7E081919D91EF012197892BB5
:104A7000888387E0E535F807B1F780911A0288232B
:104A800051F080912E028D3031F480914707809350
:104A9000540780934107DF91CF9108958EBD0DB4E7
:104AA00007FEFDCF8EB50895CF93C82FCC0FCC0F46
:104AB000289881E80E944E2585E08C0F8168CF916F
:104AC0000C944E252A9A8FE697E10197F1F700C0E2
:104AD00000002A989FE729EA83E091502040804017
:104AE000E1F700C000002A9A289882EE0E944E2525
:104AF00080EA0E944E258BEE0E944E258FE20E9496
:104B00004E2587E20E944E2589E80E944E259FEFA0
:104B100021EE84E0915020408040E1F700C0000089
:104B20008091F3010E94542584EC0E944E258FEA67
:104B30000C944E2581E58CBD0895682F70E040E40B
:104B400052E08EE592E00C94503790EC699FA00102
:104B50001124682F70E08EE592E00C945037CF93CB
:104B6000DF932898CCE3D1E4FE0184910E944E2586
:104B70002196F1E4CF34DF07B9F7DF91CF910895A3
:104B80008FE697E10197F1F700C000002A988FE6C1
:104B900097E10197F1F700C000002A9A8FEC97E0A7
:104BA0000197F1F700C000000895EF92FF921F9364
:104BB000CF93DF93162F2898806B0E944E2580E1BB
:104BC0000E944E2580E10E944E2580E00E944E25E5
:104BD000289A8EE5E82E82E0F82E20EC1203E00100
:104BE0001124C25ADD4FEC16FD0631F4DF91CF914E
:104BF0001F91FF90EF900895F70181917F010E942E
:104C00004E25F1CFCF93DF9380E00E949D25289819
:104C100080EB0E944E2580E10E944E2580E10E949B
:104C20004E2580E00E944E25289AC0E0D6E080E024
:104C30000E944E252197D9F7DF91CF9108952898AA
:104C40008EEA0C944E2528988FEA0E944E2584EA1D
:104C50000C944E25803C08F56831F8F4E62FE69573
:104C6000E695E695677090ECE99FF0011124E25A11
:104C7000FD4FE80FF11D21E030E0062E01C0220FAC
:104C80000A94EAF7209580812823A42FA17001C0FF
:104C9000AA0F6A95EAF72A2B208308950F931F9392
:104CA000CF93DF93D62FC82F840F9927991F8C019C
:104CB000C01711062CF0DF91CF911F910F9108952D
:104CC00041E06D2F8C2F0E942A26CF5FF1CF0F93EA
:104CD0001F93CF93DF93D82FC62F042F440F110BB0
:104CE000060F111D67FD1A95C01711062CF0DF91F4
:104CF000CF911F910F91089541E06C2F8D2F0E944D
:104D00002A26CF5FF1CF8052282F30E091F0F901B1
:104D1000EE0FFF1FE35BFE4B85919491F901EE0FBF
:104D2000FF1FE15BFE4B25913491922F981B892F39
:104D3000089580E0F3CF0F931F93CF93DF938C01FF
:104D4000C0E0D0E0F801ED0FF11D8081811107C0B6
:104D50008FEF8C0FDF91CF911F910F9108950E94DB
:104D600083268F5FC80FDF5FEDCF7F928F929F9278
:104D7000AF92BF92CF92DF92EF92FF920F931F9369
:104D8000CF93DF93D62EC22E8052A82FB0E0D0E072
:104D9000C0E039F0FD01EE0FFF1FE35BFE4BC59154
:104DA000D491FD01EE0FFF1FE15BFE4B85919491C5
:104DB000782E7C1A8D2C912CC40130EC439F800DF1
:104DC000911D1124FC01E25AFD4F5F01882D8D19C0
:104DD000871588F081E08D0D870DDF91CF911F91B0
:104DE0000F91FF90EF90DF90CF90BF90AF909F908A
:104DF0008F907F900895CE018A5D9E4F0E94573715
:104E0000082FCE0196958795805090400E94573785
:104E100090E0C0FBEE24E0F8F12C9701220F331F45
:104E2000220F331F02C0959587952A95E2F7182F18
:104E30001F70000F111F000F111F20EC821691042C
:104E40004CF48C2D8027F5018083E054FF4F8C2D8E
:104E500081278083FFEFAF1ABF0A21962FEF821AB6
:104E6000920AB4CFFF920F931F93CF93DF93EC017D
:104E7000042FF22E10E0FE01E10FF11D808181115F
:104E800007C0862FDF91CF911F910F91FF9008955A
:104E90002F2D402F0E94B526682F1F5FECCFEF9279
:104EA000FF920F931F93CF93DF93142FEC01649F16
:104EB000C00DD11D1124622FF12CF11208C0862FD4
:104EC000DF91CF911F910F91FF90EF900895FE0118
:104ED00084912E2D402F0E94B526682FF3942196A1
:104EE000ECCF262F2150330BF901E05DFE4BE4910E
:104EF00091E0633008F090E0891B282F26952695D5
:104F0000280F3327331F64E60E940F37B901681B4F
:104F10007109CB018E0F911D840F911D67E070E028
:104F20000E941B378F5F0895823021F4637081F4F3
:104F30008DE108958150990B67E070E00E941B3766
:104F400062E070E00E941B379FE1981B892F089553
:104F50008CE108958D3010F08C500895811101C0BE
:104F60008CE00895CF93DF93DC01362F4423C1F00A
:104F70006A30B0F4E0E0222311F02C93E1E0ED017F
:104F8000CE0FD11D832F6AE00E940F37905D98836A
:104F9000EF5FEA0FFB2FF11D1082DF91CF91089593
:104FA000832F6AE00E940F37805D8C93E7CFCF920A
:104FB000DF92EF920F931F93CF93DF9300D000D037
:104FC0000F92CDB7DEB7282F81EFC82E81E0D82E03
:104FD000F60162896150EE24EA9400E043E085EF37
:104FE00090E40E944F27682F2FEF40E08DE20E944F
:104FF000B526282FF6016285615043E08BE091E4ED
:105000000E944F27682F2FEF40E08DE20E94B526C7
:10501000182FF601638520E041E0CE0101960E9441
:10502000B2272FEF40E0612FCE0101960E94322778
:105030000F900F900F900F900F90DF91CF911F91D5
:105040000F91EF90DF90CF9008951F93CF93DF9350
:1050500000D000D00F92CDB7DEB7182F8091F601A7
:10506000813009F042C06091020220E241E0CE01AD
:1050700001960E94B2272FEF40E0612FCE010196EA
:105080000E943227682F2FEF40E08AE30E94B52666
:10509000182F6091F80120E040E0CE0101960E94B7
:1050A000B2272FEF40E0612FCE0101960E943227F8
:1050B000682F8091F601813079F48091F7012FEF0C
:1050C00040E08C30BCF080E50E94B526682F2FEFC1
:1050D00040E08DE40E94B5260F900F900F900F9046
:1050E0000F90DF91CF911F9108956091F70120E219
:1050F00040E0BDCF81E4E8CF0895EF92FF920F9397
:105100001F93CF93DF9300D000D000D0CDB7DEB790
:1051100002E010E0EE24E394F12C2091240730917A
:105120002507C701002E02C0880F991F0A94E2F7D5
:1051300082239323892BE9F0EDEFE00FE83028F488
:10514000F0E0EF59F84C0C942F376BE770E0CE018C
:1051500001960E94493720E040E060E0CE010196D0
:105160000E94322706C020E040E06BE186E60E9404
:10517000B5260F5F1F4F0B30110579F626960FB637
:10518000F894DEBF0FBECDBFDF91CF911F910F917D
:10519000FF90EF90089520E040E064E287E6E7CFDB
:1051A00065E770E0CE0101960E94493720E040E0BB
:1051B0006EE2D4CF20E040E068E587E4D8CF61E735
:1051C00070E0CE0101960E94493720E040E060E6A1
:1051D000C5CF6CE670E0CE0101960E94493720E011
:1051E00040E06BE7BBCF20E040E06BE983E4BFCF5A
:1051F00068E670E0CE0101960E94493720E040E069
:1052000067EAACCFBF92CF92DF92EF92FF920F93FB
:105210001F93CF93DF93CDB7DEB728970FB6F894DF
:10522000DEBF0FBECDBF84E0E82E82E0F82E8CEF0B
:105230008F83D12C10E000E0EF81EF5FE887CF8013
:10524000C394C394FF81F25FFD838F81835F898361
:10525000EF81E45FEE83BF80BA94FF81F75FFA834A
:105260008F81865F8B83EF81E55FEC83F70180811F
:105270009181002E02C0969587950A94E2F780FFEF
:1052800028C0EFEFE00FE83028F4F0E0E759F84CE1
:105290000C942F374BE060E08F810E944E2649E04E
:1052A00061E088850E944E2647E062E08C2D0E94D6
:1052B0004E260FC045E063E08A810E94672647E0E2
:1052C00062E08B810E94672649E061E08C810E9448
:1052D00067260F5F1F4F0930110541F6D394FF81F8
:1052E000FE5EFF8382E0E80EF11CF23C09F0A2CFE3
:1052F00028960FB6F894DEBF0FBECDBFDF91CF91D9
:105300001F910F91FF90EF90DF90CF90BF90089585
:1053100045E06DE08A810E94672647E06CE08B8162
:105320000E94672649E06BE0D1CF47E062E18C2D17
:105330000E944E2649E063E188850E944E264BE09C
:1053400064E18F81B4CF49E06BE08B2D0E9467262A
:1053500047E06CE08F810E94672645E06DE088851C
:10536000B6CF49E061E08B2D0E94672647E062E0FE
:105370008F810E94672645E063E0F1CFD1100EC017
:1053800048E069E081E00E944E264AE06AE080E061
:105390000E944E2648E06BE081E089CF49E069E059
:1053A00088850E944E264BE06AE08F810E944E263F
:1053B00049E06BE088857BCF43E062E189810E9410
:1053C0004E2643E063E189810E944E2643E064E17A
:1053D00089816DCF42E065E18D810E944E2642E0D9
:1053E00066E189810E944E2642E067E18E815FCFAF
:1053F0004F925F926F927F928F929F92AF92BF92E5
:10540000CF92DF92EF92FF920F931F93CF93DF9390
:1054100000D000D000D0CDB7DEB72EE032E0DE0104
:10542000119680E060E470E11FE00CE09BE0F92E53
:1054300049E0E42E58E0D52EE6E0CE2EF5E0BF2E72
:1054400094E0A92E4AE0942E52E0852EEEE07E2EC6
:1054500093E0FDE06F2E5524539447E0442EF9016C
:10546000419151919F01FA01EF77FF27E636F1054F
:10547000A0F4E034F10509F48FC008F071C0E933FD
:10548000F10509F48FC090F4E630F10509F474C019
:10549000379709F47BC06C930CC0E656F109EA31EA
:1054A000F105C8F7EF58F84C0C942F37FF9799F790
:1054B0001C92843011F447FD9D838F5F11968630D6
:1054C00071F61E811034A9F18D818A3091F18F70AF
:1054D0002AE0829F100D11248A819B81803409F07B
:1054E00069C0FC80392F3F70329FF00C1124DD24FD
:1054F000D3943981303408F08EC09F702AE0DC806C
:10550000929FD00C1124F82E329FF00C1124EE241F
:10551000EA9400E025E543E06F2D86E294E00E94E6
:105520004F27FAE2FF1609F44DC08BE2F81609F492
:105530005CC026960FB6F894DEBF0FBECDBFDF91DC
:10554000CF911F910F91FF90EF90DF90CF90BF9080
:10555000AF909F908F907F906F905F904F90089545
:10556000EB35F10559F0EE35F105F1F0EF34F105C9
:1055700009F091CF9C939DCF5C929BCF8C9299CF59
:10558000AC9297CFBC9295CFCC9293CF4C9291CFC7
:10559000DC928FCFEC928DCF9C928BCFFC9289CFF7
:1055A0000C9387CF6C9285CF7C9283CF1C9381CF55
:1055B0007C937FCF382F3F70F92E329FF00C11244F
:1055C000D12C97CFEE24EA9400E021E843E06D2D42
:1055D00088EF92E00E944F27E6E1DE1213C025EA31
:1055E00043E0612F86E294E02FC0EE24EA9400E0CD
:1055F00021E843E06D2D8FE893E00E944F27F6E10C
:10560000DF1669F3EE24EA9400E025EA43E0612F17
:105610008FE792E019C0EE24EA9400E09034F8F6A7
:105620002FE6D11021E843E06F2D86E294E00E943E
:105630004F278AE2F8120BC0EE24EA9400E025EA34
:1056400043E0612F88EF92E00E944F2772CFEBE298
:10565000EE24EA9400E025EA43E0612F8FE893E02E
:10566000FE1691F3D110D4CFEDCFE62FE69547E0AB
:10567000489F9001499F300D112429553B4FE20F5F
:10568000F32FF11D808160FD82958F7008952F9218
:105690003F924F925F926F927F928F929F92AF92C2
:1056A000BF92CF92DF92EF92FF920F931F93CF930F
:1056B000DF93CDB7DEB728970FB6F894DEBF0FBEE5
:1056C000CDBF2091A0042B8330914F023A833090BC
:1056D000310284E0882E82E0982E18861F8219827B
:1056E000B12CA12C66246394712C4F818AE0463042
:1056F00008F489E05B81552309F497C09A819923C6
:1057000019F0332009F491C0F3010F8002C0EE0FAD
:10571000FF1F0A94E2F7FD83EC8394E14F815885E3
:10572000949F9001959F300D1124F901E050FF4F97
:105730007F01D12CC12C10E000E0482E512CCE82EC
:10574000F7012180222099F06081C2010E94352B4F
:10575000282269F0F9E0CF1609F462C0C3010C2CCD
:1057600002C0880F991F0A94E2F7082B192B3FEF0C
:10577000C31AD30A42E0E40EF11C5AE0C516D10464
:10578000F1F6F401808191818017910711F0F1E029
:10579000F983F401019311934F01809124079091B3
:1057A00025078A159B0519F0F981F260F983B092FB
:1057B0002507A09224072F8138852F5F3F4F388718
:1057C0002F832B30310509F090CF3A81332371F0CC
:1057D0008091A10481508093A104811107C081E0D0
:1057E00083258093310284E18093A10489812896E6
:1057F0000FB6F894DEBF0FBECDBFDF91CF911F91E2
:105800000F91FF90EF90DF90CF90BF90AF909F905F
:105810008F907F906F905F904F903F902F90089562
:105820002C813D81A22AB32AA2CF10E000E0A9CFAB
:105830009C01211588E1380760F0305245EF54E0B3
:10584000E5EFFAE0211588E1380738F080E090E0D4
:10585000089545EF52E2E5EFF8E2E20FF31F84917D
:105860008227F901F695E795F695E795E40FF51F80
:10587000449150E02370220F02C0559547952A9518
:10588000E2F7942F93700895CF93DF93FC01DB012F
:10589000241718F4DF91CF910895842F90E0ED0143
:1058A000C80FD91F38818E0F9F1FEC0138834F5FBF
:1058B000EFCF9C01461708F40895F901E60FF11D9A
:1058C00010826F5FF7CF4DE060E084E397E00E94C5
:1058D000592C4DE060E080E592E00E94592C4DE0AB
:1058E00060E087E497E00C94592C282F22952F70C4
:1058F00051F08091480290914902807F822B9093D1
:105900004902809348024DE060E087E497E00E94FE
:10591000592C80914802909149029C012F7E283099
:10592000310531F44DE060E087E497E00C94592CA8
:105930008B31910510F0855A910927E0289FD001FD
:10594000299FB00D1124A955BB4FE7E4F7E08D91D5
:10595000982F9F70908382958F708183329687E015
:10596000E535F807A1F70895CF93DF93DC01CB016C
:10597000241718F4DF91CF910895E42FF0E0ED01A2
:10598000CE0FDF1F3881E80FF91F50815883308315
:105990004F5FEECF2DE040E065E577E087E497E0EC
:1059A0000C94B42C2DE040E06DE172E087E497E0C8
:1059B0000C94B42CCF93DF93EC01DB01022E000C8E
:1059C000330B51E0642F70E0261737071CF4DF918A
:1059D000CF91089590E0109721F0FD01E60FF71F99
:1059E0009081FE01E60FF71F808160913D02860FD6
:1059F000890F90914607891730F0891B50933D021B
:105A000080834F5FDFCF10923D02FACF0F93CF9389
:105A1000DF93FC01DB01BA0131E0021724F4DF91CE
:105A2000CF910F91089580E0109731F0ED01C20FF2
:105A3000D11D27FDDA95888190E06115710531F05F
:105A4000EB01C20FD11D27FDDA95988140913D02EF
:105A5000841B891B87FF0FC090914607890F3093E5
:105A60003D02309731F0EF01C20FD11D27FDDA95CD
:105A700088832F5FD2CF10923D02F3CF9C0146174F
:105A80000CF40895F901E40FF11D47FDFA95461352
:105A900003C010824150F3CFDF0111978C918083B6
:105AA000F9CF9C0146170CF40895F901E60FF11D9A
:105AB00067FDFA95641303C010826F5FF3CF818195
:105AC0008083FBCFFC01CB0110923D0224170CF424
:105AD0000895642F042E000C770B30E0009721F01E
:105AE000DC01A60FB71F3C916E0F7F1F51E0DB0159
:105AF0006C91631301C050E030913D02352B30931F
:105B00003D024F5FE3CF282FFB014AE0642F0E9444
:105B10000F37382F905D9283243660F00E940F3744
:105B2000805D8083832F6AE00E940F37905D9183B0
:105B30001382089580E280832A30A0F78183F8CF12
:105B4000F89410924D0210922D0210923B02109286
:105B5000450778940895F89490913B029730ECF4BF
:105B6000E0912D02F0E0E05CFD4F808380912D02FA
:105B70008F5F80932D0280912D02877080932D027C
:105B800080913B028F5F80933B0280913B02877044
:105B900080933B0281E0809345077894089561509B
:105BA00086230895262F30E0082E000C990BB901AA
:105BB0000E941B37820F931FB9010E941B37089563
:105BC00087FD8195089585E880937A008EE680931D
:105BD0007C0087EC90E00197F1F700C00000809115
:105BE0007A00806480937A0080917A0086FDFCCFF1
:105BF00010927A00809179000895682F8091DE01DB
:105C0000883628F02FEF40E085E70C94B5260895FC
:105C100062E08FEF0E94A5258091240790912507CF
:105C200092FF10C080914F0281110CC082E00E944F
:105C300025288FE30E94FD2D0E94F82962E080E074
:105C40000C94D52582E00E94D7278A5F0E942528E0
:105C500086EB0E94FD2D8091F8018093E001EECF4C
:105C6000282F80918000211104C08F7780938000BD
:105C70000895806880938000022E000C330B2F5F04
:105C80003F4F4FEF429FC001439F900D11246AE0A8
:105C900070E00E941B37709389006093880008951C
:105CA000F89480913B021816BCF4E0914D02F0E0AC
:105CB000E05CFD4F808190914D029F5F90934D027B
:105CC00090914D02977090934D0290913B029150AC
:105CD00090933B02789408958FEFFCCF8091420718
:105CE000811104C08091A004882359F08091A204FE
:105CF0009091A304009731F001979093A3048093AF
:105D0000A204089580913A028130C1F0823001F1FD
:105D10008111F7CF0E94502E8F3F99F3E82FF0E0CA
:105D2000E354FB4FE491E0931B0281E08093EC018C
:105D300080933A028091FE0190E0DFCF8091450789
:105D4000882321F080913B021816DCF682E0F0CF28
:105D50001092EC0110921B0210923A02EBCF0E94BB
:105D60006E2E81E09091EC01911101C080E0809352
:105D70003D0208950C946E2EFF920F931F93CF93C4
:105D8000DF93C82FF62E082F10E08B3009F04DC09E
:105D90006091FA018091FB010E949427F801EA5E6C
:105DA000FD4BD491D801AF50BE4F2C914F2D0F2CED
:105DB000000C550B240F352F311D82171306D4F517
:105DC000DC934091FC016091FB018091FA010E94FB
:105DD0007127809303028091F7010E94AA27809384
:105DE00002021091FC016091FA018091FB010E9476
:105DF0009427212F110F330B8217130644F460915F
:105E0000FA018091FB010E9494278093FC01C2302B
:105E1000D1F1D8F4C11121C08091F101DF91CF916E
:105E20001F910F91FF900C94302EF801EB5FFD4B0A
:105E30008491B4CF4D2F0D2E000C550B2417350730
:105E400014F48C93BECF2C93BCCFC33029F1DF91D7
:105E5000CF911F910F91FF9008959091F201809141
:105E6000F4011F144CF4891710F4D093F2018091BF
:105E7000F20180933C02EBCF8917C8F78091F401BF
:105E80008093F201F4CF8091F301DF91CF911F91C4
:105E90000F91FF900C9454259091F2018091F401A0
:105EA0008917A8F68091F4018093F201D0CF2F9248
:105EB0003F924F925F926F927F928F929F92AF929A
:105EC000BF92CF92DF92EF92FF920F931F93CF93E7
:105ED000DF9300D000D00F92CDB7DEB762E080E054
:105EE0000E94A525E12C00E027E046E060E08FE37A
:105EF00092E40E944F272CE54AE060E084E392E4BC
:105F00000E944F2762E080E00E94D52562E080E099
:105F10000E94A52520E048E060E084E792E40E942A
:105F20004F2762E082E00E94D52562E080E00E9477
:105F3000A52520E046E160E08DE592E40E944F2730
:105F400062E084E00E94D52562E080E00E94A52501
:105F500020E046E160E086E492E40E944F2762E0A0
:105F600086E00E94D5252FE73AE186E021503040B7
:105F70008040E1F700C00000809145078111ABC06F
:105F800000E010E095E4892E24E3622E31E3532EE5
:105F900040E3442E992493945CE0F52E01112AC12C
:105FA000A12EA594A594A89CA02C1124D12CC12C81
:105FB000812F8370282E62E080E00E94A5253C2C72
:105FC0002C1006C020E040E06A2D84E70E94B52630
:105FD000BC2CE12C00E028E044E06C2D8DE792E43D
:105FE0000E944F27F601EF50FE4F8081BE016F5F88
:105FF0007F4F0E94832D20E040E06BE2CE010196AE
:106000000E9432272DE444E064E06C0D8DE792E4B9
:106010000E944F277C2C770CF601EB50FE4F91E04D
:1060200093150CF460C06081670D20E743E087E2C0
:1060300092E40E944F2768E06B0DE12C00E022E91A
:1060400044E08DE792E40E944F27F601E750FE4FAF
:106050008081BE016F5F7F4F0E94832D20E040E072
:1060600061EBCE0102960E94322762E0872D0E94EA
:10607000D5252FEFC21AD20A34E0C316D10409F095
:106080009ACF9092E1018091E101813029F48091D1
:106090003B02882309F456C08091A404811173C087
:1060A00082E08093A4040F900F900F900F900F90B8
:1060B000DF91CF911F910F91FF90EF90DF90CF90E4
:1060C000BF90AF909F908F907F906F905F904F9018
:1060D0003F902F9008959FE728E331E091502040B2
:1060E0003040E1F747CF8081BE016F5F7F4F0E9454
:1060F000832D20E040E060E7CE0102960E94322727
:106100009ACF198220E040E060E7CE0101960E941C
:10611000322762E08B2D880F0E94D525B3948FEF34
:10612000C81AD80A01E094E0B91271C0AACFBE0122
:106130006F5F7F4F8091DE01AAC06B8259824A82D5
:106140001C82E0CF8091800087FF19C083B7817FD8
:1061500083BF25E02093B1008091B6008F71E1F7F5
:1061600083B7816083BF889583B78E7F83BF80911B
:106170004507813009F087CF1092E10184CF83B7C2
:10618000817F8660E5CF0E94502E90914507911146
:106190000FC08832B8F4803208F496C0E0EEE80F01
:1061A000E83008F091C0F0E0E557F84C0C942F3738
:1061B0003FE798E321E0315090402040E1F700C0F4
:1061C0000000E3CF8F3F09F0E9CE3FE788E391E09D
:1061D000315080409040E1F700C00000DFCE1F5FEB
:1061E000011105C01C3009F0DBCE10E0D9CE133010
:1061F00008F010E0A12EA594A594A89CA02C112431
:106200008CE0C82ED12CB12C812F8370782E62E0C7
:1062100080E00E94A5257B1006C020E040E06A2DAA
:1062200084E70E94B526E12C00E028E044E06C2DD4
:106230008DE792E40E944F27F601EF50FE4F8081D8
:10624000BE016F5F7F4F0E94832D20E040E06BE234
:10625000CE0101960E9432272DE444E060E16B0DEF
:106260008DE792E40E944F2792E0B91609F45FCFC0
:1062700023E0B21609F461CF31E0B31609F441CF3F
:10628000F601EB50FE4F8081BE016F5F7F4F0E9491
:10629000832D38CF115008F081CE1BE0002309F484
:1062A0007FCE12E0A7CF6FEF812F0F9D800D1124BD
:1062B0000E94BC2E73CE61E0F7CF66EFF5CF6AE0A7
:1062C000F3CF092510E06ACE8A3109F4ECCE66CE10
:1062D00080E00E94302E1092680088E087B94398D1
:1062E000E0E8F0E080818F7780830E941F26109283
:1062F000690081E08DBB0895CF93C9B1C6FBCC275F
:10630000C0F981E0C82780E04A998F5FE7ECF0E0B0
:106310003197F1F700C000008F3FB1F787B918B887
:106320008091F20180933C028091F1010E94302E15
:106330000E94A02D8AE10E94AB2D84E0809368002A
:106340008C2FCF910895FF920F931F93CF93DF93DC
:106350008091E101811156C0FF24F394C1E0D0E0A7
:1063600080914B0290914C02029709F051C08091AC
:10637000EA019091EB019093EF018093EE018091FF
:10638000EE019091EF010E94182CAC0160913D024A
:1063900060931A0210923D0220914B0230914C0200
:1063A0002230310509F4A7C1C0F58091A504909170
:1063B000A604232B09F050C19A01369527953695EE
:1063C0002795FC013196F093A604E093A504742F61
:1063D00073707230B1F1733009F42DC1713031F145
:1063E000F901FF27EE0FFF1FE158FF4F4591549130
:1063F000822FFA01099580914B0290914C02892BD2
:1064000009F0AECFDF91CF911F910F91FF900895CA
:106410008091A5049091A604AECF2330310509F4F4
:106420006DC110924C0210924B02E5CFD0934C02FA
:10643000C0934B0250933F0240933E026093E601AB
:10644000DACF122F169516951695E22FE770E150C8
:10645000E73040F4F0E0ED56F84C0C942F372DE087
:1064600060E005C00E94A221FC016081262F2093DC
:106470002E0211501F31F0F4E12FF0E0E656F84CF7
:106480000C942F370E94A221FC012081E9CF60915A
:10649000ED0120914407261754F72DE0E8CF22E0C4
:1064A00062E0E5CF2CE063E0E2CF2DE06DE0DFCFEE
:1064B00022E0D6CF422F84E397E00E94592C9BCF55
:1064C000422F80E592E0F9CF422F87E497E0F5CFA5
:1064D000462F60E572E084E397E00E94B42C8BCFF6
:1064E000462F64E377E080E592E00E94442C83CF5E
:1064F000462F67E477E0EFCF462F60E572E087E450
:1065000097E0F3CF462F67E477E080E592E0E5CFB0
:10651000462F67E477E084E397E0E7CF462F60E516
:1065200072E084E397E00E94DA2C65CF462F67E49F
:1065300077E0F7CFF0923D02462F70E060E0F1CFB8
:10654000022F262F40E552E064E377E0CB010E9462
:10655000062D51CFF0923D02022F262F50E040E051
:10656000F3CF022F262F47E457E0EECF462F67E404
:1065700077E0CB01D8CF462F64E377E087E497E05C
:10658000D2CFF0923D02462F70E060E0F7CF022FAD
:10659000262F47E457E064E377E0CA01D8CFF092B2
:1065A0003D02022F262F50E040E067E477E0CECF97
:1065B000F0923D02022F262F47E457E070E060E0A2
:1065C000ECCF462F70E060E080E592E00E94622D03
:1065D00012CF462F70E060E087E497E0F7CF022FFC
:1065E000262F47E457E064E377E090E080E0AFCF08
:1065F000022F262F40E552E0F6CF462F70E060E0F4
:1066000084E397E0E3CF462F67E477E0F9CF422FAA
:1066100084E397E00E94512DEECE422F80E592E078
:10662000F9CF422F87E497E0F5CF422F84E397E03C
:106630000E943E2DE0CE422F46954F7327FD4054D9
:1066400021702613D8CE840F911D47FD9A95909303
:10665000A6048093A504CFCE9C012F5F3F4F3093BB
:10666000A6042093A50410924C0210924B02609154
:10667000E601CA01817099276817190609F0BBCE97
:1066800080913E0290913F029695879596958795C9
:10669000BA01E6E0660F771FEA95E1F76627862BD9
:1066A000972B41FDD4CF4091360250913702509341
:1066B0003902409338024091340250913502509390
:1066C0003702409336024091320250913302509388
:1066D0003502409334023093330220933202909378
:1066E000A6048093A5040E94182C892B09F083CE60
:1066F0000E94DB21ACCF0E94C3237DCE8091A504F4
:106700009091A60401969093A6048093A504CA01D3
:106710000E94C32370CE1F920F920FB60F921124C6
:106720002F933F934F935F936F937F938F939F9399
:10673000AF93BF93CF93DF93EF93FF938091E101EA
:10674000823091F08091A404882371F08091A40498
:1067500081508093A4048091A404811105C01092FB
:10676000E1018AE10E94AB2D80913C02882309F46B
:1067700073C080913C02815080933C028091F9016A
:106780008F5F8093F9018091F9018C330CF451C033
:106790001092F9010E94E32D8091F8018F5F8093A0
:1067A000F8018091F8018C330CF443C01092F80189
:1067B0008091F7018F5F8093F7018091F701883115
:1067C00094F11092F7018091FC018F5F8093FC019E
:1067D000C091FC016091FA018091FB010E94942715
:1067E0000C2E000CDD0B8C171D069CF491E0909391
:1067F000FC018091FB018F5F8093FB018091FB0185
:106800008D303CF09093FB018091FA018F5F809373
:10681000FA014091FC016091FB018091FA010E9414
:106820007127809303028091F7010E94AA27809329
:106830000202FF91EF91DF91CF91BF91AF919F91B4
:106840008F917F916F915F914F913F912F910F9019
:106850000FBE0F901F90189580E00E94302E8ECFB3
:106860001F921FB61F9211248F931DBA1092E1013F
:106870008091F4018093A4048F911F901FBE1F90FC
:1068800018951F921FB61F9211242F933F934F9379
:106890008F939F9380914507813059F58091DF0157
:1068A00081508093DF018091DF01811122C08091AE
:1068B000FF018093DF0149B180919E0490919F0474
:1068C000880F991F21E030E04F3F11F430E020E0C5
:1068D000822B932B90939F0480939E0480919E041F
:1068E00090919F04892B29F41092450784E08093AE
:1068F00068009F918F914F913F912F911F901FBEE4
:106900001F9018951F920F920FB60F9211242F937C
:106910003F934F935F936F937F938F939F93AF9327
:10692000BF93EF93FF9349B14F3F71F130E020E007
:1069300061E070E0822FFB01022E01C0EE0F0A948D
:10694000EAF7E7B995E39A95F1F7000099B1941742
:1069500031F02F5F3F4F2530310561F785E030E0A2
:1069600020E050E0622FFA01022E02C0F595E79573
:106970000A94E2F7E0FF1DC02F5F3F4F2930310539
:1069800089F78FEF87B918B88091F4018093A40438
:10699000FF91EF91BF91AF919F918F917F916F91F7
:1069A0005F914F913F912F910F900FBE0F901F90CD
:1069B0001895853031F3283021F33D9A9FEF30E26E
:1069C0002091F501222319F028B1232728B9E3EFFC
:1069D000F1E03197F1F700C00000915089F79091F4
:1069E0003B029730F4F4E0912D02F0E0880F880F1D
:1069F000880F860FE05CFD4F808380912D028F5FB2
:106A000080932D0280912D02877080932D028091BA
:106A10003B028F5F80933B0280913B0287708093A3
:106A20003B021092680081E090E090939F04809375
:106A30009E048091F20180933C028091F1010E94BA
:106A4000302E8091E101813011F41092E10181E05A
:106A5000809345079091FF019093DF018093420757
:106A600090CF8FE284B98FEF87B91AB88BB918B875
:106A700080936D0084E08093680014BC15BC16BC44
:106A800084B5826084BD85B5826085BD81E487BDA3
:106A9000EEE6F0E0808182608083A0E8B0E01C92A6
:106AA000E1E8F0E01082109285001092840081E00D
:106AB0008C9380831092B00085E08093B100E0E772
:106AC000F0E0808181608083E6EBF0E0808180628D
:106AD000808381E58CBD0FB6F894A8958091600005
:106AE000886180936000109260000FBE78940895D2
:106AF0000E9431350E94622587E38093F9018BE380
:106B00008093F8011092F7018CE080930202C5E0B7
:106B1000C093FC0183E08093FB0185E18093FA013F
:106B20004091FC016091FB018091FA010E94712764
:106B3000809303028FEF8093E00181E08093F60160
:106B400084E08093F3011092F1011092F501C0935B
:106B5000F2018CE38093F40180E18093FD018AEFE0
:106B60008093000288E28093FE018AE08093FF0117
:106B70000E94A02D8091F20180933C028091F1014E
:106B80000E94302E8091F3010E9454258091F401DF
:106B90008093A4040E9402260E94E32DE7EAF4E019
:106BA0001082118212821382148215821682379605
:106BB00027E0E432F207A1F781E0809342071092C8
:106BC000A6041092A50480933D02E4E3F7E020E5DB
:106BD00032E087E497E0C5E5D7E06DE172E042E49A
:106BE00057E01192D9011D929D01DC011D92CD014A
:106BF0001992DB011D92BD014E175F0791F71092AC
:106C00002B0210922C021092E70110923002109287
:106C10002F021092ED011092440710921C0280E1A5
:106C20008093460710924C0210924B0210923A0247
:106C300019E1D5E0C1E08091000280934E0280917D
:106C4000FD01819FC00111249093E5018093E4012F
:106C50000E946E2E0E94A3318091E4019091E50183
:106C600001979093E5018093E40120914E02215019
:106C700020934E02892B61F70E94472B9091DD01F2
:106C8000892B8093DD0180FF0EC080E00E949D254E
:106C90000E94022963E083E00E94D5258091DD01F6
:106CA0008E7F8093DD018091DD018695813089F4AE
:106CB00062E080E00E94A5250E947D2862E086E0D7
:106CC0000E94D5258091DD018D7F8093DD010E949A
:106CD000082E8091E101823009F04BC00E9402260B
:106CE0000E9468318091E101823009F482C00E94E3
:106CF0002326BFE72AE186E0B15020408040E1F73B
:106D000000C000000E9423260E947C31813079F46B
:106D10000E94502E8F3FE1F70E94572F0E94A02D16
:106D20008AE10E94AB2D1092E1010E9402260E948E
:106D3000022963E083E00E94D5250E94E32D809321
:106D4000DE010E94082E8091F8018093E001C0933B
:106D500042071092A6041092A50410924C021092C1
:106D60004B02C0933D0210923A02C093A0041092CD
:106D70004F0280913A0281115ECF80913B028111D6
:106D80005ACF809145078091680082FF54CF80914F
:106D9000E101813009F04FCF80914F0281114BCF3B
:106DA0008091800087FF37C083B7817F83BFD093F6
:106DB000B1008091B6008F71E1F783B7816083BF26
:106DC000889583B78E7F83BF9091F8018091E00111
:106DD000981751F00E94E32D8093DE010E94082E47
:106DE0008091F8018093E0018091E1018130C1F24E
:106DF00022CF83B7817F866083BFD093B10080911B
:106E0000B6008F71E1F783B7816083BF889583B740
:106E10008E7F83BF67CF83B7817F8660C7CF991B83
:106E200079E004C0991F961708F0961B881F7A9581
:106E3000C9F78095089597FB072E16F4009407D0A4
:106E400077FD09D00E94353707FC05D03EF49095B8
:106E500081959F4F0895709561957F4F0895EE0F2E
:106E6000FF1F0590F491E02D0994AA1BBB1B51E173
:106E700007C0AA1FBB1FA617B70710F0A61BB70BAA
:106E8000881F991F5A95A9F780959095BC01CD014F
:106E90000895FB01DC0105900D920020E1F70895B3
:106EA000DC0101C06D9341505040E0F70895F9991D
:106EB000FECF92BD81BDF89A992780B50895F894C8
:106EC000FFCFB328CB28D028DA28DF28E928F328F9
:106ED000F8285A2988299529A329B129BE29DC290E
:106EE000EA29C02A4B2A4B2A4B2A4B2A4B2A4B2AE7
:106EF000C22A4B2ACA2A4B2AD82A4B2A4B2A4B2A67
:106F00004B2A4B2ACE2A4B2AD62A4B2A4B2AD02A46
:106F1000C42A4B2AC82A5B316431613153315D3157
:106F20004A315F31EF30583242322F3247324F32DE
:106F300052325532603264326832703278327C328A
:106F4000823288328E3296329A32A032AA32B132EE
:106F5000B632BB32C132C732CF32DA32D832E13246
:106F6000E932EF32F832FD32033307330D33113398
:026F70001533D7
:106F72000000000000000000000000000B04000000
:106F8200000000000502050804080B0804040501BE
:106F920005040908090400000608070206020402A3
:106FA2000601060407010308030404010C080D028C
:106FB2000C0203020C010C040D010D080D04030167
:106FC2000802080807080202070408010804090267
:106FD200090102010A080B020A0201080A010A0455
:106FE2000B01020802040104020803020202030860
:106FF200020102040301040204010304050205085C
:10700200040801080404050105040602060101043E
:10701200070207080608090806040701070409020F
:10702200090109040B080C020B0208020B010B04F4
:107032000C010808080408010D020D080C080A02D8
:107042000C040D010D040A080A040A0101015D0A7B
:00000001FF
